:020000040800F2
:104000000040002099420008119A00082974000815
:104010006589000839580008A1D700080000000091
:10402000000000000000000000000000AD4100089A
:10403000755B00080000000035420008854200085A
:10404000B3420008B3420008B3420008B34200087C
:10405000B3420008B3420008B3420008915C000874
:10406000995C0008B3420008B3420008B34200085C
:10407000B3420008B3420008B3420008B34200084C
:10408000B3420008B3420008B3420008B34200083C
:10409000B3420008B3420008B3420008A15C000824
:1040A000B3420008B3420008B3420008B34200081C
:1040B000B3420008B3420008B3420008B34200080C
:1040C000B3420008B3420008B3420008B3420008FC
:1040D000B34200089DCC0008A5CC0008ADCC000878
:1040E000B3420008B3420008B3420008B3420008DC
:1040F000B3420008B3420008B3420008B3420008CC
:10410000B3420008B3420008B3420008B3420008BB
:10411000B3420008B3420008B3420008B3420008AB
:10412000B3420008B3420008B3420008B34200089B
:10413000DFF80CD000F0B2FD0048004789E5000828
:104140000040002080F309887047EFF30980704732
:10415000684680F3098804480078C00714BF02202D
:10416000032080F314887047D4FA0008DFF818C0E1
:10417000EFF305831B0618BF6047EFF31483DB07DB
:1041800008BF604700DF704791ED0008DFF818C0F6
:10419000EFF305831B0618BF6047EFF31483DB07BB
:1041A00008BF604700DF704739EF0008EFF3098070
:1041B000816911F8021C39BB90E80F10E047EFF35A
:1041C000098C194B93E80600914218D059B10CB4F0
:1041D0004FF0010381F826302CE9F00FC1F82CC014
:1041E0000BF0D4F80CBC1A60D2F82CC0BCE8F00F6D
:1041F00092F826308CF309881BB192F82500CCF890
:1042000000006FF0020E704710B5084A1268914224
:1042100009D8074C54F8214090E80F10A047EFF35D
:10422000098C8CE80F0010BD680100204850000880
:10423000485000080AF05EFF114B93E806009142D7
:104240001BD00CB44FF0000381F82630EFF3098C3B
:104250002CE9F00FC1F82CC00BF098F80CBC1A60D8
:10426000D2F82CC0BCE8F00F8CF3098892F8263005
:104270001BB192F82530CCF800306FF0020E704779
:10428000680100200BF054F9D6E700000AF062FA4A
:104290000BF04EF9D0E7000006488047064800477B
:1042A000FEE7FEE7FEE7FEE7FEE7FEE7FEE7FEE7E6
:1042B000FEE7FEE7F5C300083141000840EA0103CC
:1042C0009B0703D009E008C9121F08C0042AFAD2CC
:1042D00003E011F8013B00F8013B521EF9D2704790
:1042E000D2B201E000F8012B491EFBD27047002238
:1042F000F6E710B513460A4604461946FFF7F0FFE5
:10430000204610BD421E12F8013F002BFBD111F8D0
:10431000013B02F8013B002BF9D1704730B505464F
:104320002A460B4612F8010B13F8014B08B1A042C4
:10433000F8D01CB1002802D06D1CF1E7284630BD32
:1043400010B5044604E00B7800F8013B03B1491CAA
:10435000521EF8D2204610BD421C10F8011B002945
:10436000FBD1801A704730B504460020034600E0B8
:104370005B1C934203D2E05CCD5C401BF8D030BDA7
:10438000034611F8012B00F8012B002AF9D1184639
:1043900070472DE9F0410E460546002400E0641CFC
:1043A000285D00F058FB0746305D00F054FB381ADA
:1043B00002D1295D0029F2D1BDE8F0810FB400B52A
:1043C0008DB010A909900B9000914FF0FF300A902A
:1043D00000200C9005480690054807906A4609A8F9
:1043E0000F9900F053FB0DB05DF814FBA94A0008CB
:1043F000C74A00082DE9FF5F1D464FF0FF3BD5E996
:10440000014691465F464FF00008A9697F1C01985C
:104410008847296A824688470028F6D11AF10100A8
:104420000CD024F4C064002E19DD600614D5BAF156
:104430002B0F09D0BAF12D0F0ED103E0584604B06E
:10444000BDE8F09F44F48064A9697F1C0198884707
:10445000761E8246002E02DDBAF1300F03D0B9F18C
:10446000000F26D032E0761EA96944F400747F1C48
:10447000019888478246002E05DDBAF1780F06D0F4
:10448000BAF1580F03D0B9F1000F10D01EE0B9F106
:10449000000F02D0B9F1100F18D1761EA96924F4CB
:1044A00000747F1C019888478246102002E0082093
:1044B00000E00A20814609E008FB0908761EA96988
:1044C00044F400747F1C019888478246002E05DD65
:1044D0004946504600F0C5FA0028EDDAE96901982E
:1044E0008847A00502D46FF00100A8E7E00727D1B4
:1044F000600614D5600502D5C8F1000000E0404612
:10450000296801F104022A600968220501D50870B2
:1045100016E0220701D5088012E0086010E0286844
:1045200000F1040129600068210502D580F80080AF
:1045300006E0210702D5A0F8008001E0C0F8008065
:1045400038467CE72DE9F04791460F468046044601
:10455000002614F8015B2DB100F070FA0068405D90
:10456000C007F6D12B2D02D02D2D18D0641E4A463F
:104570003946204600F0B8FA27B13968A14201D186
:10458000C7F8008071054FF002040BD540420028A7
:1045900003DD09F0AFFA0460A007BDE8F08746F438
:1045A0008066E4E70028F8DA09F0A4FA04606FF006
:1045B0000040F2E770B5064609F09CFA046805462B
:1045C0000A2200213046FFF7BDFF2C6070BD70B598
:1045D000064609F08FFA046805460A220021304693
:1045E000FFF7B0FF2C6070BD2DE9FE4F804681EAD9
:1045F0000300C00F0C46009021F0004123F000455D
:10460000B8EB0200A94105D24046214690461C461F
:104610000B46024623F00040104304D14046214699
:1046200003B0BDE8F08F270DC7F30A00C3F30A51AA
:104630000290401A0190402866DAC3F3130040F458
:10464000801B0098924620B10023D2EB030A63EB53
:104650000B0B01985946C0F14002504600F0BDF9DD
:1046600006460D4650465946019A00F0D5F910EB22
:1046700008006141002487EA115284EAE7731A4373
:104680003BD0009A3AB3019A012A4FEA075210DC54
:10469000001B61EB02014FF0004202EA0752CDE934
:1046A0000042001C41F5801132462B4600F078FA9A
:1046B000B6E7001B61EB0201001C41F580130018F6
:1046C0005B412018A2F5001747EB030140EAD570C3
:1046D000B6196D4111E06D084FEA360645EAC0751E
:1046E0004FEA0752001B61EB0201001C41F58011EB
:1046F00049084FEA30000019514132462B4603B0B9
:10470000BDE8F04F00F03FBA0098012240000023BE
:10471000D0EB020263EBE073009821464FEAE074AD
:10472000B8EB000061EB0401E9E783F000435BE7CD
:1047300081F0004158E72DE9FE4F81EA030404F0BF
:10474000004421F0004100944FF0000B23F000439F
:1047500050EA010402D052EA030404D100200146C9
:1047600003B0BDE8F08FC3F30A54C1F30A552C44DB
:10477000A4F2F3340194A0FB0254C1F3130141F4F9
:104780008011C3F3130343F4801301FB024400FBC5
:10479000034E840A970A44EA815447EA8357A4FBEC
:1047A000076802958D0A05FB07854FEA932C04FBE9
:1047B0000C542705029D4FEA065847EA1637B5EB19
:1047C00008056EEB070C870E920E47EA811742EA46
:1047D0008312A7FB0201B6EB0B0164EB00042B0D67
:1047E00043EA0C335E1844EB1C50DA465146E7FBB3
:1047F0000201C5F313044FEA0B3343EA14534FEAA3
:104800000432019C43EA0603A4F10C040294009CC8
:10481000CDE900B400F0C4F9A2E72DE9F04D81EA3A
:10482000030404F0004B21F0004514464FF0000A49
:1048300023F0004150EA050220D054EA01021DD0C5
:10484000C5F30A570246C5F31303C1F31300C1F3BE
:104850000A5640F4801543F48013A7EB0608101B9A
:10486000D64608F2FD3873EB050002D308F10108C3
:1048700001E092185B41B8F1000F03DA0020014615
:10488000BDE8F08D00204FF48011064684460EE00E
:10489000171B73EB050705D3121B63EB05030643D8
:1048A0004CEA010C49084FEA300092185B4150EA8B
:1048B0000107EDD152EA030012D082EA040083EA34
:1048C0000501084303D100224FF0004308E0101B0C
:1048D000AB4102D20122002302E06FF0010253102B
:1048E0001AEB06004CEB085110EB0A0041EB0B01F0
:1048F000BDE8F04D00F047B90EB5C10F80EAE07099
:104900000844CA07002140F233438DE80E000A46EE
:104910000B4600F045F903B000BDC1F30A5210B5D3
:10492000C1F3130140F2FF3341F480119A4201DADE
:10493000002010BD40F233439A42A2F2334203DC1E
:10494000524200F059F810BD904010BD30B50B46F2
:10495000014600202022012409E021FA02F59D42AF
:1049600005D303FA02F5491B04FA02F52844151E83
:10497000A2F10102F1DC30BD2DE9F05F0546002017
:1049800092469B4688460646814640241BE02846C0
:1049900041464746224600F02FF853465A46C01A71
:1049A000914110D311461846224600F016F82D1AF0
:1049B00067EB01084F4622460120002100F00DF868
:1049C00017EB00094E41201EA4F10104DFDC48462C
:1049D00031462A464346BDE8F09F202A04DB203AB0
:1049E00000FA02F1002070479140C2F1200320FA42
:1049F00003F3194390407047202A04DB203A21FA40
:104A000002F00021704721FA02F3D040C2F12002E7
:104A10009140084319467047202A06DBCB17203AFD
:104A200041FA02F043EAE07306E041FA02F3D040B3
:104A3000C2F1200291400843194670470048704770
:104A4000C4FB000810B50446FFF7F8FF0068005DDE
:104A500000F0010010BDA0F14101192900D820305B
:104A600070473A2800D2303820F02002412A01D382
:104A7000A2F13700884201D34FF0FF3070470000A9
:104A8000026811441378016018467047D1600449E8
:104A900051610449116200211161114600F010B901
:104AA000814A0008454A0008426842B1016811F88D
:104AB000013B23B1521EC0E9001218467047012184
:104AC000C160881E704742685AB1C368016843B923
:104AD00083688B4205D0491E521CC0E90012002099
:104AE00070474FF0FF3070472DE9F05F8246007845
:104AF000002715468B460AF10104B946302801D03B
:104B00009DB113E014F8010B0127782803D0582831
:104B100001D045B10AE00DB1102D07D100271025B5
:104B200014F8010B02E0082500E00A250026B04633
:104B30000EE005FB080005FB06F1012701EB10461E
:104B40001FFA80F8B6F5803F00D3B94614F8010B80
:104B50002946FFF786FF0028EBDABBF1000F05D0EE
:104B60000FB1641E00E05446CBF80040B9F1000FCD
:104B700006D008F0BFFF02210160C81EBDE8F09F0B
:104B800048EA0640FAE710B5002B08DA401C41F16C
:104B9000000192185B411A4301D120F0010010BDC1
:104BA0002DE9F04D92469B4611B1B1FA81F202E037
:104BB000B0FA80F220329046FFF70FFF04460F460E
:104BC00040EA0A0041EA0B0153465A46084303D122
:104BD00020463946BDE8F08D114653EA010015D054
:104BE000C8F140025046FFF707FF05460E46504603
:104BF00059464246FFF7F1FE084301D0012000E08C
:104C00000020054346EAE0762C4337430A984FEAF2
:104C10004453A0EB08004FEAD4240A304FF00002BE
:104C200044EA47544FEAD72502D500200146D1E790
:104C3000010510196941DDE9084500196941BDE820
:104C4000F04DA0E7C1F30A52C1F3130140F2FF3364
:104C500041F480119A4202DA00200146704740F286
:104C600033439A42A2F2334202DC5242FFF7C4BEFF
:104C7000FFF7B3BE30B5002904DB4FF000444042DB
:104C800064EB0101002B04DB4FF00044524264EB63
:104C90000303994208BF904230BD0000064C074D07
:104CA00006E0E06840F0010394E8070098471034FC
:104CB000AC42F6D3FFF740FA74FC000894FC0008FD
:104CC0002DE9F34F8BB04FF0000801F10C000C46BA
:104CD0004FF0010B46460DF1080A0190626901216F
:104CE0000198904705002DD0252D2CD0216A8847AA
:104CF000C0B16269012101989047216A8847002864
:104D0000F7D1411E62690198904700E0761CA169C5
:104D10000B988847216A88470028F7D1E1690B98EA
:104D20008847DBE7A1690B9888470746A84201D16D
:104D3000761CD3E7E1690B9888477F1C02D1B8F154
:104D4000000F6FD045E1002762693D463946019862
:104D500090472A2804D162690121019890470125D2
:104D6000DFF884926269012101989047A0F1300137
:104D70000A290AD24F45E5DC07EB870100EB410722
:104D8000303FDFD445F01005ECE7E90601D46FF0C1
:104D900000476C280AD04C2814D0682815D06A28FF
:104DA0000DD074281CD07A281AD01DE06269012128
:104DB000019890476C2802D045F0040514E045F0B6
:104DC00002050DE045F020050AE062690121019825
:104DD0009047682802D045F0080505E045F40065D5
:104DE0006269012101989047C4E9015765283DD0C7
:104DF00019DC582879D00CDC452837D004DC25286C
:104E000026D0412831D131E046282FD047282CD157
:104E10002CE05B287FD0612828D063287BD06428D1
:104E200023D159E0CFE06F2847D008DC66281DD099
:104E300067281BD0692821D06E2816D127E070285A
:104E400044D0732867D0752846D078280DD14CE01F
:104E5000A1690B988847054625283FF469AFE169A9
:104E60000B9888476D1C3FF46AAFB2E023466A4650
:104E70006FF001000B99AFF300809DE045F040001A
:104E80006060A80723464FF0000235D43DE020685B
:104E900000F1040121600068290501D506701DE7B5
:104EA000290701D5068019E7A90704D54FEAE6715D
:104EB000C0E9006112E7066010E745F0400060605D
:104EC000A80723464FF0080216D41EE040F60E0154
:104ED00025EA0100606016E045F040006060A80728
:104EE00023464FF00A0207D40FE045F0400060600F
:104EF000A80708D5234610226FF001000B99AFF3E5
:104F0000008059E007E0234610226FF001000B9962
:104F1000FFF770FA50E04FF000094F464B46632808
:104F200002D05B2806D040E0E80601D40120A06052
:104F300001273AE062690121019890475E2805D176
:104F40004FF001096269494601989047216939B9D2
:104F500000210B46524642F82130491C0829FADB51
:104F6000B0B3216969B9C11700EBD1614B110AEBEC
:104F7000830221F01F01411A012013688840034376
:104F8000136062690121019890475D28E8D1B9F169
:104F9000000F09D00020514651F82020D24341F89B
:104FA0002020401C0828F7DB02AB224600976FF058
:104FB00001000B99AFF3008000280CDA401C08D1E7
:104FC000BBF1000F05D04FF0FF300DB0BDE8F08F02
:104FD000FFE74046F9E7E90701D108F10108064477
:104FE0004FF0000B7AE60000CCCCCC0C70B501EB96
:104FF000020410F8015B15F0070301D110F8013B22
:105000002A1106D110F8012B03E010F8016B01F80A
:10501000016B5B1EF9D12B0705D40023521E0FD460
:1050200001F8013BFAE710F8013B02F10202A1EBA3
:10503000030303E013F8015B01F8015B521EF9D58D
:10504000A142D6D3002070BD0000000000B587B09B
:105050000121480205F078FF0121082005F074FFC6
:105060000120ADF8040000208DF8070001A91248C6
:1050700001F0F8F9002002908DF80C008DF80D0079
:105080004FF4602004900020059001208DF8180056
:1050900002A90A4800F02CF800230122194607480B
:1050A00000F04EF80121054800F00AF801210348FC
:1050B00000F0A2F807B000BD000801400024014044
:1050C00021B1826842F00102826003E0826822F02E
:1050D0000102826070470146C86C80B27047024688
:1050E000002013680B4201D0012000E0002070472F
:1050F00030B502460020002350680F4C20400D7947
:105100000C6844EA05242043506090680B4C204012
:10511000D1E902542C434D7944EA45042043906080
:10512000D06A20F470000C7C641EE4B2234340EA91
:105130000350D06230BD0000FFFEF0FFFDF7F1FF2D
:10514000F0B504460D4600200021092D11DDE06870
:10515000A5F10A0606EB4607072606FA07F188437B
:10516000A5F10A0606EB460603FA06F10843E060DD
:105170000CE0206905EB4507072606FA07F188438E
:1051800005EB450603FA06F108432061072A0FDA0A
:10519000606B561E06EB86071F2606FA07F188434A
:1051A000561E06EB860605FA06F10843606322E008
:1051B0000D2A0FDA206BD61F06EB86071F2606FA8C
:1051C00007F18843D61F06EB860605FA06F1084369
:1051D000206310E0E06AA2F10D0606EB86071F26A9
:1051E00006FA07F18843A2F10D0606EB860605FADA
:1051F00006F10843E062F0BD21B1826842F4A002EA
:10520000826003E0826822F4A0028260704700009E
:105210002DE9F04104460A46254610E008F1010058
:1052200000F0FF0803F00F071E11304600F037F8BA
:1052300002F8010B384600F032F802F8010B15F8BD
:10524000013B002BEAD104480078B8EB400FE5DBC6
:1052500000201070BDE8F081B00000202DE9F0477B
:1052600006460C4637464FF0040811E017F8015B7C
:1052700005F00F0A4FEA2519484600F010F804F827
:10528000010B504600F00BF804F8010BA8F10108DF
:10529000B8F1000FEAD100202070BDE8F0870028A7
:1052A00005DB092803DC00F13001C8B208E00A2858
:1052B00005DB0F2803DC00F15701C8B200E0FF2036
:1052C000704700002DE9F04196B0044650227F4916
:1052D00002A8FEF7F3FF7EA1204604F03FF830B9A4
:1052E000204601F0BDF9804608F014FAEBE07AA1FF
:1052F000204604F033F830B9204601F0B7F9804673
:1053000008F008FADFE076A1204604F027F828B973
:10531000204601F0F5FB75494870D4E074A12046A1
:1053200004F01CF838BB754800780228DED0012153
:10533000204601F007FB71480078012810D10121B7
:10534000204601F0FFFA69498870084680780228F3
:10535000CCD16B48807820F0080069498870B2E0B1
:10536000664800780028C1D1604880780128BDD106
:1053700064490870A7E064A1204603F0EFFF00280D
:1053800059D10120034655A20D210090204600F07E
:1053900090FF0546B0F1FF3FA8D06019FFF70AF96A
:1053A000C7B2012003465BA20D210090204600F009
:1053B00080FF0546B0F1FF3F98D06019FFF7FAF87B
:1053C00086B20220012353A20D210090204600F056
:1053D00070FF0546B0F1FF3F75D0012F24D147483B
:1053E000007820B96019314602F048F86BE0434874
:1053F0000078012867D1605D7E280FD1A819401E72
:10540000205C7E280AD1711E6A1CA01809F094FC49
:1054100086B26019314602F043FF54E001223EA1FA
:10542000002006F0A7FF4EE0022F4CD16019314654
:1054300002F024F847E03DA1204603F08FFF00BBB7
:10544000607A4F2802D1A07A4B2808D0607A412890
:1054500039D1A07B642836D1E07D742833D1274828
:10546000007830B9012027490870002032490870BF
:1054700029E022480078012802D11C49887022E0E6
:1054800021E02EA1204603F069FFE0B12FA12046C4
:1054900003F064FF70B91948007850B9A07A312838
:1054A00011D11848007802280DD000201549087045
:1054B00009E008E028A1204603F050FF18B90120B8
:1054C000284981F8300116B0BDE8F081ECFA0008F7
:1054D0002B434353513A00002B4353513A000000F1
:1054E0002B504F435F5050503A000000EB0000201B
:1054F0002B5443505354415455533A001C0100203F
:10550000B01D0020150100202B5443505245435636
:105510003A0000002C000000556E6B6E6F776E2015
:1055200050726F746F636F6C000000002B54435017
:105530004F50454E3A000000130100202B544350B9
:10554000434C4F53453A4F4B000000002B544350FF
:10555000434C4F53453A00002B504F433A5354416C
:1055600052540000D827002010B5A2B0012215A186
:10557000002006F0FFFE1C2102A8FEF7B8FE154829
:10558000016802918188ADF80C1080798DF80E00C9
:10559000142211490DF10F00FEF790FE1B20009020
:1055A0000E48D0F81D1002AB4FF4817209A807F025
:1055B00059F884B2224609A9012002F04BFE22B01C
:1055C00010BD000041757468656E7469636174692B
:1055D0006F6E2100F9180020103500204C180020B3
:1055E00000B589B00121042005F08EFC01210920BD
:1055F00005F0AAFC8020ADF8200018208DF82300CB
:1056000003208DF8220008A91B4800F02BFF212160
:10561000072006F0F7F942F21070ADF818000320E9
:10562000ADF814000020ADF81A00ADF816008DF8A2
:105630001C0005A9114806F09FFF7020ADF804007A
:1056400041F28830ADF80A000120ADF806000220D2
:10565000ADF80C0001A9094806F02EFF0821074803
:1056600006F07CFF3421072006F0CCF90020044925
:10567000086009B000BD0000000C014000080040B7
:105680002000002010B51B4890F893101AA008F0D5
:10569000F9F9184890F89300062828D2DFE800F0BE
:1056A00003090F151B21012216A1032003F024F981
:1056B0001EE001221FA1032003F01EF918E00122C1
:1056C00028A1032003F018F912E0012231A10320E0
:1056D00003F012F90CE001223AA1032003F00CF9C7
:1056E00006E0012246A1032003F006F900E000BF16
:1056F00000BF10BD4C180020675F6E65743D2564C7
:105700000D0A00003531374644433745424538429B
:1057100036453746304346463533354634443532D0
:1057200035313746444337454541383141383532C4
:1057300000000000353137463231364142453842AB
:1057400036453746304346463533354634443532A0
:1057500038433445323139453231364130463546A9
:10576000000000003531374632313641424538427B
:105770003645374630434646353335463444353270
:10578000303934453231394532313641304635468B
:105790000000000035313746444337454245384222
:1057A0003645374630434646353335463444353240
:1057B0004442353632313945454138314138353248
:1057C00000000000353137464443374542453842F2
:1057D0003645374630434646353335463444353210
:1057E0004442353632313945333130303338303058
:1057F0003330303033303030343635310000000053
:1058000035313746444337454245384236453746B9
:1058100030434646353335463444353244423536D6
:105820003231394533383030333030303330303046
:10583000343635310000000004480268044801880D
:1058400004A008F01FF900BFFEE700004800002098
:10585000460000200D0A5B4246485D463D25642C0B
:105860004C3D25640000000010B53148007800B9B7
:1058700010BD30480078401CC0B22E490870102876
:105880000CDD2D480078012805D100202A49087038
:1058900028490870ECE7002026490870274800785E
:1058A000401CC0B2254908700A283EDD24484078D3
:1058B000012837D120480078002833D120480078CB
:1058C000F8B92048006818B11E480068632819D14B
:1058D00001201D4908600A214FF4936006F0D0FAB8
:1058E0006E20DFF868C000DF0120174908600A2138
:1058F0004FF4936006F0C4FA012215A1002006F0CF
:1059000039FD0FE00F48006801280BDD0D480068E5
:10591000632807DA01200C4908600C214FF49360DA
:1059200006F0AEFA00200549087000BFA0E70000AD
:10593000F80000202A0000206A00002068000020F3
:10594000D8270020C0000020140C0140E5EE00081C
:105950004353515F50726F6D70742E2E2E2E2E2E6B
:105960002E2E2E0070B58CB004460E4630220CA1AF
:105970006846FEF7A3FC2E2C01D10A2509E0302C45
:1059800005DB392C03DCA4F13000C5B201E00CB01A
:1059900070BD684600EB85000068306000BFF6E728
:1059A0004331453344324242423646454338464409
:1059B00043424334434545354331463943364446F3
:1059C00042304342424543354235453300000000F2
:1059D00010B50446B4F5A57F0DDA012211A100200F
:1059E00006F0C8FC00201549C87220201449086040
:1059F00006F062FC15E0B4F5AA7F0FDA11480078D2
:105A0000401CC0B20F4908701E280ADD0020087033
:105A100000220DA1012002F06FFF02E000200949E1
:105A2000087010BD56626174206C6F7721736875C1
:105A300074646F776E206E6F77210000D827002086
:105A4000140C014064000020433745424233453482
:105A5000423545370000000010B5044624B1012C42
:105A60001AD0022C62D13DE0012231A1002006F0C3
:105A700081FC0A20DFF8C4C000DF31480470012235
:105A800040F225512F4807F0BEF9002240F2244190
:105A90002C4807F0B8F949E000F0D8FD01222AA10E
:105AA000002006F067FC0A20DFF890C000DF2448E1
:105AB0000470012240F22551224807F0A4F9002287
:105AC00040F224411F4807F09EF9012240F225517F
:105AD000224807F098F9002240F224411F4807F0BD
:105AE00092F923E001221EA1002006F043FC0A20C7
:105AF000DFF848C000DF12480470012240F225514F
:105B0000104807F080F9002240F224410D4807F0C8
:105B10007AF9012240F22551154807F074F9002264
:105B200040F22441124807F06EF900BF00BF10BDDB
:105B3000434F4D3C2D2D3E4D43552100E5EE0008D1
:105B40000400002000380140434F4D3C2D2D3E4DB8
:105B50006F64656D5F4750532100000000480040AE
:105B6000434F4D3C2D2D3E4D6F64656D210000006F
:105B700000440040704770B5044626466B2107205C
:105B800005F040FF01F020FE09E0002501E0681C5F
:105B900085B241F270708542F9DB01F015FE3000EC
:105BA000A6F101018EB2F0D17121072005F02AFF84
:105BB00070BD000010B50024022000F0A5F818B157
:105BC0000124022000F08EF8042000F09DF818B1A6
:105BD0000224042000F086F81CB32948006810F065
:105BE000040F06D02748007840F0010025490870CE
:105BF00005E02448007820F0010022490870204880
:105C0000006810F0020F06D01E48007840F0020035
:105C10001C49087005E01B48007820F00200194973
:105C200008701848007800F00300012802D002280C
:105C30001FD10FE014480078032803D10120134935
:105C4000088006E01048007818B94FF0FF300F497F
:105C500008800EE00C48007818B901200B49088034
:105C600006E009480078032802D1001F0749088090
:105C700000BF00BF034800780349087010BD000052
:105C8000080C0140000000200100002092000020CC
:105C900010B5FFF78FFF10BD10B5FFF78BFF10BDDC
:105CA00010B54FF4007000F023F801280DD107481B
:105CB0000078012805D12020054908600120054908
:105CC00008704FF4007000F007F810BD300000209D
:105CD000100C0140310000200149086070470000AD
:105CE0001404014001490860704700001404014099
:105CF00001460020034A12680A4201D0012000E058
:105D00000020704714040140014600200022074B88
:105D10001B6803EA0102054B14331B680B4202D0D7
:105D20000AB1012000E0002070470000000401409B
:105D3000002123498279002A3AD00A461268036872
:105D40009A430B461A600A1D126803689A430B1D9A
:105D50001A60027911440A6803681A430A60184AF3
:105D60000832126803689A43154B08331A601A1DEB
:105D7000126803689A43124B0C331A604279102A56
:105D80000ED11A1F126803681A430D4B08331A60AC
:105D90001A1D126803681A43094B0C331A600DE090
:105DA0000749427911440A6803681A430A6005E00A
:105DB000027911440A6803689A430A607047000038
:105DC000000401400EB504208DF80B0003208DF86F
:105DD0000A000620ADF8080002A9104800F042FBB6
:105DE0000220FFF77FFF0420FFF77CFF0121084618
:105DF00000F018FB0221012000F014FB06200090A7
:105E000000208DF8040010208DF8050001208DF889
:105E100006006846FFF78CFF0EBD0000000C014035
:105E200000B589B08A48008808B909B000BD884823
:105E3000B0F90000002814DD8648007800280CDD49
:105E400085480068002802DA0020834908608248FB
:105E50000068401C804908601CE000207E49086002
:105E600018E07B48B0F90000002813DA7948007880
:105E700000280CDD78480068002802DD0020764903
:105E8000086075480068401E7349086002E0002001
:105E900071490860DFF8C4C100DF714909688842B0
:105EA00003D200206A490880BFE7DFF8B0C100DFF5
:105EB00032306B4908606648B0F9000000285CDDAC
:105EC000012268A1002006F055FA674800780228F0
:105ED00012D166480078052805D100206349087072
:105EE0005B490880A1E761480078401C5F49087061
:105EF00000205749088098E75D48007870B102207B
:105F00005B49087001205B4908605BA003F094F9CD
:105F100001225EA1002006F02DFA93E05E48007891
:105F20000028FAD002205C4908705C48008A40B919
:105F300000205A494882002259A1012002F0DCFCCD
:105F400008E05648428A5EA101A807F0BFFD01A8FB
:105F500003F072F95148408A401C50494882084673
:105F6000408A098A884202DB00204C49488201228B
:105F700059A1002006F0FEF964E0012259A1002099
:105F800006F0F8F938480078022812D1374800782E
:105F900030B905203549087000202D49088044E7B4
:105FA00032480078401E3149087000202849088096
:105FB0003BE72F48007870B102202D49087001207E
:105FC0002C49086048A003F037F901224BA10020BA
:105FD00006F0D0F936E030480078002832D00220B0
:105FE0002D4908702D48008A40B900202B4948826D
:105FF00000222BA1012002F07FFC08E02748428A02
:106000002FA101A807F062FD01A803F015F92348AC
:10601000408A002805DD2148408A401E1F494882E9
:106020000BE01E48008A18B900201C49488204E091
:106030001A48008A401E19494882012232A10020D4
:1060400006F098F900200249088000BFEDE6000044
:1060500092000020370000203C00002071F500086D
:106060005C0000205B2B5D00280000206900002000
:1060700034000020140C014041542B504F433D315B
:10608000303030303030370D0A0000005B47726F1F
:1060900075702B2B5D00000035000020D8270020F4
:1060A00043454445433645344342464342334339EE
:1060B00044344231443444414346444600000000E5
:1060C00041542B504F433D31303030303032312548
:1060D0003034780D0A0000005B557365722B2B5D20
:1060E000000000005B2D5D0041542B504F433D31BB
:1060F000303030303030380D0A0000005B47726FAE
:1061000075702D2D5D0000005B557365722D2D5D42
:106110000000000010B5002019490870012019493D
:1061200008600A214FF4936005F0AAFE1420DFF8FE
:1061300058C000DF0120134908600A2140F26E3088
:1061400005F09EFE1420DFF840C000DF01200D495D
:1061500008600A214FF4936005F092FE01200B497C
:10616000087006F053FF012001F008FF082005F039
:10617000B9FF012206A1002006F0FCF810BD0000C6
:10618000F8000020140C0140E5EE00080500002096
:106190005B456E74657254784D6F64655D000000F8
:1061A00030B5044604254FF4302000F06FF8054662
:1061B000042D17D10C48006940F002000A4908611B
:1061C00008464461006940F0400008614FF4302007
:1061D00000F05CF805460448006941F6FD7108408E
:1061E00001490861284630BD0020024004200B49C7
:1061F000C96811F0010F01D001200EE00749C968FC
:1062000011F0040F01D0022007E00449C96811F021
:10621000100F01D0032000E004207047002002404E
:106220000348006940F080000149086170470000A0
:106230000020024070B504460D460426F00200F02E
:1062400025F80646042E11D10948006940F00100E6
:10625000074908612580F00200F018F80646044856
:10626000006941F6FE71084001490861304670BD81
:1062700000200240024803494860034848607047D4
:106280002301674500200240AB89EFCD00B50246EF
:106290000423FFF7ABFF034603E0FFF7A7FF034626
:1062A000521E012B01D1002AF7D102B9052318464D
:1062B00000BD2DE9F04704460E4617461D46DDF8A1
:1062C00020A04FF00008C14615E02A463946204676
:1062D000FEF749F850B909F1010000F0FF09D14576
:1062E00004D108EB050000B2BDE8F087641C08F19A
:1062F00001001FFA80F82078B042E6D14FF0FF305D
:10630000F2E7000010B501F05FFA3748007800B9F5
:1063100010BD3648407840B33448007800BB34485C
:106320000078C0EB001084003048C07B401CC0B235
:106330002E49C873A04218DD0020C87301222DA188
:1063400006F018F805F048FB2E480078401CC0B253
:106350002C490870022808DD0020087006F07AF841
:1063600000202249C873274908702048C07A0128B4
:1063700021D11E48807B10B90020234908701B489A
:10638000807B401CC0B219498873232813DD00208C
:10639000887301221DA105F0EDFF05F01DFB1A48D1
:1063A0000078401CC0B218490870022803DD0020A4
:1063B000087006F04FF81A48007800F00100002835
:1063C0000FDD17484078401CC0B2154948700A28B4
:1063D00007DD0020487000F039F907F007F906F0F2
:1063E0002BF900BF94E70000F8000020D827002018
:1063F00043000020506F634C6F737454696D656F78
:106400007574210065000020660000204D6F6465F2
:106410006D5265637654696D656F75742100000077
:10642000B01D002030B500228B071C0F0F2303FA8C
:1064300004F20B4B8C1053F824309343084C8D100E
:1064400044F8253023468C1053F824308C07240F51
:1064500000FA04F42343024C8D1044F8253030BD7B
:10646000080001402DE9F0410246002500260020E9
:1064700000230024002791F803C00CF00F0591F8C9
:1064800003C01CF0100F03D091F802C04CEA0505C0
:1064900091F800C0BCF1000F31D0146800202BE04F
:1064A0004FF0010C0CFA00F3B1F800C00CEA03063F
:1064B0009E4220D183004FF00F0C0CFA03F7BC432F
:1064C00005FA03FC4CEA040491F803C0BCF1280F60
:1064D00006D14FF0010C0CFA00FCC2F814C00AE01F
:1064E00091F803C0BCF1480F05D14FF0010C0CFA34
:1064F00000FCC2F810C0401C0828D1D31460B1F8C9
:1065000000C0BCF1FF0F34DD546800202EE000F124
:10651000080C4FF0010808FA0CF3B1F800C00CEABF
:1065200003069E4221D183004FF00F0C0CFA03F7B3
:10653000BC4305FA03FC4CEA040491F803C0BCF127
:10654000280F05D100F1080C08FA0CF8C2F81480E5
:1065500091F803C0BCF1480F07D100F1080C4FF0CF
:10656000010808FA0CF8C2F81080401C0828CED3A5
:106570005460BDE8F0810000F0B50A460023002415
:106580000021002500F00046B6F1004F02D11D4E5B
:10659000F16901E01B4E7168C0F3034583B200F45A
:1065A0004016B6F5401F08D121F07061154E76688F
:1065B00026F07066134F7E6012E000F48016B6F588
:1065C000801F06D1032606FA05F4A14341F070614D
:1065D00006E0460D360103FA06F6B14341F070615C
:1065E00022B1460D360103FA06F6314300F00046AB
:1065F000B6F1004F02D1034EF16101E0014E71602E
:10660000F0BD0000000001400246002093680B42EC
:1066100001D0012000E000207047000008B51020E4
:106620008DF8030003208DF802004FF48040ADF890
:10663000000069460448FFF715FF4FF48040024907
:106640001431086008BD0000000C01400020024920
:1066500008800249088070471A0000201C000020B2
:1066600010B50446E01DFDF7A5FF10BD10B50446AA
:10667000A01DFDF79FFF10BD2DE9F04FCBB0804668
:106680008A4693464FF4807233490BA8FDF716FEF5
:106690003248824503D200204BB0BDE8F08F584607
:1066A000FDF75AFE07460E2F03D00F2F01D0002012
:1066B000F2E752462AA108A807F008FA08A8FDF751
:1066C0004BFE00900025A7F10A0405E01BF804002A
:1066D00004A948556D1C641CBC42F7DB0026B1467A
:1066E000002407E008A8005D464004A8005D80EA99
:1066F0000909641C0A2CF5DB86EA09060BA810F8C8
:10670000069000240CE008A8005D80EA090604A8B1
:10671000005D704001A908550BA810F80690641C94
:106720000A2CF0DB002504240FE001A8005D0A21FB
:1067300090FBF1F201FB120008F8050018F80500C3
:10674000303008F805006D1C641C0A2CEDDB0020BD
:1067500088F8060001209FE7C4F900082058F208D5
:10676000253031306C7500002DE9F04F9BB00020D2
:10677000189019901A90159002F080F816A96B489D
:10678000FEF76CFD00201490002404E016A8005DC4
:1067900014A90855641C032CF8DB14A8FDF70AFFA4
:1067A0000E90002011901290002405E016A9E01C24
:1067B000085C11A90855641C062CF7DB11A8FDF72D
:1067C000F9FE81464FF47A7099FBF0F00590FEF7E0
:1067D00093F8CDE90C010022554BDDE90C01FEF7E1
:1067E0001CF8CDE90C014FF47A7099FBF0F100FB35
:1067F0001190C0EB001080000590FEF77DF8CDE908
:106800000A0100224B4BDDE90A01FEF706F8CDE94B
:106810000A01DDE90A23DDE90C01FDF7E5FE054685
:106820000E460022444B28463146FDF784FFCDE951
:106830000201424A0E9901FB02F0FEF75DF8CDE934
:106840000001DDE90223FDF7CFFECDE90401FEF7EB
:1068500064F83B49086615A93448001FFEF7FEFCA2
:10686000002404E015A8005D13A90855641C032C3E
:10687000F8DB13A8FDF79EFE8346002405E015A96A
:10688000E01C085C0FA90855641C062CF7DB0FA858
:10689000FDF790FE82464FF47A709AFBF0F0059077
:1068A000FEF72AF8CDE908010022214BDDE90801B5
:1068B000FDF7B3FFCDE908014FF47A709AFBF0F1D0
:1068C00000FB11A0C0EB001080000590FEF714F84B
:1068D000CDE906010022174BDDE90601FDF79DFF1A
:1068E000CDE90601DDE90623DDE90801FDF77CFEBF
:1068F000074688460022104B38464146FDF71BFFED
:10690000CDE902010D490BFB01F0FDF7F5FFCDE9E3
:106910000001DDE90223FDF767FECDE90401FDF783
:10692000FCFF074948661BB0BDE8F08F983800208F
:1069300000004E4040774B4180842E4140420F0082
:10694000B01D00202DE9F04104460D46022604F159
:106950000B00FDF72FFEC7B2607B312800D1012666
:10696000AF4202D13046BDE8F0810220FBE70000D3
:1069700000B53A480078401CC0B238490870012878
:1069800001DD002008703548007820B901F0A8FA30
:106990003349086003E001F0A3FA32490860304847
:1069A000006830490968884201D0002000BD2E48A7
:1069B00000682B490968884213D0294800682A4991
:1069C0000860274800680F2806D001202749087072
:1069D00000202749087004E0002024490870254958
:1069E00008702248007858B32348007888B12348BB
:1069F00000781E490978884209D01C4800781F4950
:106A00000870194800681E4908600120CEE7002080
:106A1000CCE716480078194908701A48007840B940
:106A20000F48006816490860642016490870012064
:106A3000BCE714480078401E124908700020B5E7F2
:106A40000020104908700D48007820B100200B4943
:106A50000870401EAAE70020A8E70000950000206B
:106A60009C000020A000002098000020960000203C
:106A70008D0000208C0000208F0000209700002057
:106A8000A40000209400002000B589B010481149EE
:106A9000097800EB8100104991F89310435C0FA234
:106AA0001E2101A806F0FEFF01A802F0C5FB01228D
:106AB00001A9002005F05EFC0DA21E2101A806F030
:106AC000F1FF012201A9002005F054FC09B000BD2E
:106AD0002CF90008F90000204C18002041542B4DDF
:106AE0004F444F445245583D25640D0A00000000B4
:106AF00048414841484148414841410D0A00000091
:106B00000146487A31280CD101200B4A907010467A
:106B10004068401C5060062801D9082050600120C0
:106B2000704705484068401C034A5060062801D958
:106B3000082050600220F3E7D82700202DE9F04F0D
:106B400087B082460E4617464FF000090024A34640
:106B50009AF8000008B1307818B9002007B0BDE8F5
:106B6000F08F0FE058460BF1010B01A901F80080EE
:106B7000B8F13D0F02D0B8F13B0F01D10020EDE795
:106B8000761C641C96F80080B8F1000F01D0142C1C
:106B9000E8DB3D222046641C01A90A540020085568
:106BA0005046FDF7BBFB0546254405E028783870C4
:106BB0006D1C7F1C09F101092878202805DD287843
:106BC0003B2802D0B9F1280FF0DB0020387048468E
:106BD000C4E73EB55824684600F010F8002503E0ED
:106BE0001DF8050044406D1C0C2DF9DB04B9582438
:106BF000FF2C00D1852420463EBD00000021064A1E
:106C000000BF05E013780370401C521C4B1CD9B226
:106C10000C29F7DB70470000E8F7FF1F2DE9F0476C
:106C200007460C462046FDF797FB00F0FF08B8F139
:106C3000070F02DBB8F10F0F02DD0120BDE8F0877E
:106C40000026B246A14600251DE0605D2E2810D129
:106C5000042E08DA4846FDF7ADFCC2B23046711C7E
:106C6000CEB23A5401E00220E8E7681C04EB0009C8
:106C700007E0605D302802DB605D392801DD03201C
:106C8000DCE7681CC5B24545DFDB052E07DA484660
:106C9000FDF790FCC2B23046711CCEB23A540020CF
:106CA000CCE70000F0B589B0074617B9002009B05D
:106CB000F0BD06A8FFF7A2FF1BA006F0E3FE00242C
:106CC00006E006A8015D1BA006F0DCFE601C04B215
:106CD0000C2CF6DB19A006F0D5FE052408E03002E6
:106CE00040EA15662D0206A8005D0543601E04B249
:106CF000002CF4DAB6B22A46334611A006F0C2FEE2
:106D000013A2102102A8CDE9005606F0CBFE002404
:106D100004E002A8005D3855601C04B20F2CF8DBBB
:106D20000020F8730120C2E753544D333220494408
:106D30003D3D000025303278000000000D0A0000C3
:106D400074656D703D253031356C6C750D0A000031
:106D5000253031356C6C75002DE9F0438FB0022180
:106D60003248FEF7BCF988B13048FEF7B4F9064660
:106D700001212E48FEF740FA642E0ADAB6F5805F4C
:106D800007DB4FF0FF300FB0BDE8F0834FF0FF306E
:106D9000F9E727482749096840F821602548006835
:106DA000401C24490860092801DD002008600024F7
:106DB00006E01F4850F8240005A941F82400641C8F
:106DC0000A2CF6DB002419E000204DF824000025F1
:106DD0000DE005A850F825005DF82410884205DD77
:106DE00005A850F825004DF824002F466D1C0A2DEB
:106DF000EFDB002005A941F82700641C042CE3DB2D
:106E0000DDE9010100EB01080298C82802DA4FF021
:106E1000FF30B8E74FF49A7108FB01F0C11700EB9F
:106E200011514FEA21394846ADE7000000240140E6
:106E3000881900206000002070B594B005460E4609
:106E4000282210490AA8FDF739FA24220D492831D1
:106E500001A8FDF733FA002406E001A850F8240049
:106E6000A84200DD02E0641C0A2CF6DB00BF092CFE
:106E700000DD09240AA850F824103046FDF780FAF6
:106E800014B070BDE0F8000870B504460D461F2C24
:106E900001DC012C04DA0FA12846FDF771FA18E095
:106EA000192C04DD12A12846FDF76AFA11E0112C15
:106EB00004DD14A12846FDF763FA0AE00A2C04DD7C
:106EC00015A12846FDF75CFA03E018A12846FDF756
:106ED00057FA70BD3243303045303635353137469C
:106EE00044433745453134464637353300000000CA
:106EF00045313446463735333833384633413546E5
:106F000000000000453134464637353330323930E1
:106F100032443445000000004531344646373533AD
:106F2000344635303445344600000000453134469F
:106F300046373533383835463331354600000000A2
:106F400030B589B05248007803281CDD514880785C
:106F500020F002004F49887000204D49087001223E
:106F60004DA101A806F0B2FD01A802F065F90220CA
:106F70004E4988700020464908704648807820F0C5
:106F80000200444988704A480068632808D047488E
:106F90008078012804D13F488078C0F3400020B9B0
:106FA00000204449088009B030BD3A48016B416374
:106FB000C16A0163816AC162416A8162806935493F
:106FC0004862002404E03348243050F82450641C04
:106FD000052CF8DB0520B5FBF0F52E4805620F20E7
:106FE000354908802B488078C0F3C000F0B9334899
:106FF0000078401CC0B2314908700F2815DD002010
:1070000008702C4908802E48007870B12D4800780F
:10701000401CC0B22B490870032804DD0020087012
:1070200004F0A6F901E0FEF79FFABCE718480078E3
:1070300020B9002021490870154908701548807949
:10704000401C144988710846807810F0010F10D058
:10705000084680791C4991F8A610884216DB00206A
:107060000C498871012219A105F084F905F098FBFB
:107070000CE0084880793C2808DB0020054988712D
:10708000012218A105F076F905F076FC00BF8AE729
:1070900002000020B01D002041542B544350434CAB
:1070A0004F53453D25640D0A00000000EB00002011
:1070B000C0000020D6000020D4000020C80000201E
:1070C000D8270020D2000020E01800205453477039
:1070D0007354696D696E6753656E64506F732031C8
:1070E0003500000048656172745469636B000000EC
:1070F0002DE9F04192B004463CB100208D49086072
:107100008D49087012B0BDE8F0818C4800880028D5
:1071100005DD8B4807F0ECFD002088490880DFF88A
:1071200024C200DF83490968884200D2EAE7DFF819
:1071300014C200DF64307F490860FFF701FF824816
:107140008078032827D181480078401CC0B27F494D
:1071500008700A2822DD002008707D48807820F021
:1071600002007B49887000207A49087001227AA1C8
:1071700005A806F0ABFC05A802F05EF802207249F3
:1071800088700020734908707148807820F00200F0
:107190006F49887002E000206C49087066480078EA
:1071A000401CC0B264490870042801DD002008704A
:1071B00061480078002831D16C480078012806D158
:1071C00000206A4908706AA002F036F805E0012044
:1071D0006649087069A002F02FF86B480068FDF757
:1071E0008BFB05460022694BFDF717FB07466848F5
:1071F0000068CDE9007102905548807800F00103E5
:1072000053488078C0F3C00262A105A806F05EFC76
:10721000012205A9002005F0ADF889E04648007874
:10722000012803D164A002F007F881E04248007809
:10723000022817D156480068632800D162E7424807
:107240004078012808D101225FA105A806F03EFC84
:1072500005A801F0F1FF6BE0012260A1002005F01C
:1072600089F865E034480078032848D14848006828
:10727000632800D146E73648007810F0010F12D19C
:107280003148C078322809DA2F48C078401CC0B293
:107290002D49C870022801DB0A20C870012253A1C1
:1072A000002005F067F828488078012840D026485B
:1072B000407801283CD152480078012838D1244830
:1072C000807820F00200224988704E48C189C27D32
:1072D000807D4C4B5B7DCDE90030CDE902214948F2
:1072E000037D012248A105A806F0F0FB002205A9B4
:1072F000104605F03FF805A801F09EFF18E00E4883
:107300000078042814D122480068632800D1F9E6E7
:107310000D48807801280BD10D488078C0F34000DB
:1073200030B90B48807820F00200801C0849887032
:1073300000BFE7E6E4000020E80000201A0000207B
:10734000A80E002071F50008EB000020E9000020E5
:10735000B01D00200200002041542B544350434CE8
:107360004F53453D25640D0A00000000D100002068
:1073700041542B4353510D0A0000000041542B434C
:107380004353510D0A0000002C000020000059401A
:10739000C00000205B4154485D25642C5B4750537E
:1073A0005D25642C5B4241545D25302E32662C5B9A
:1073B0004353515D2564000041542B504F435F50AF
:1073C00050500D0A0000000041542B5443505354B8
:1073D000415455533D25640D0A00000057616974FE
:1073E00020504F435F505050000000004750532042
:1073F0006D6F64656D206E6F7420776F726B210006
:107400001C010020E018002041542B5443504F50E1
:10741000454E3D25642C25642E25642E25642E259D
:10742000643A25640D0A00000748007810B107A0EF
:1074300006F028FB0A4802680A4801880AA006F0FC
:1074400021FB00BFFEE700001E000020466C6173B8
:1074500068436865636B204661696C65640D0A006A
:1074600048000020460000200D0A5B4846485D4663
:107470003D25642C4C3D25640D0A00002DE9F04F9C
:10748000B5B0064689463446002006907748007815
:1074900030B176480078022802D035B0BDE8F08FD0
:1074A00014F8018B14F8017B4FF6FF7000EA0727F0
:1074B00007F47F4714F8010B0743F81C484506D032
:1074C0006BA107A806F002FB01200690BCE04FF07C
:1074D000000A002505E0705D504400F0FF0A681CBA
:1074E00085B2B81C8542F6DBA9F10100305C50453D
:1074F00006D061A107A806F0E9FA02200690A3E0F1
:10750000B8F1120F09D0B8F1190F06D05CA107A885
:1075100006F0DCFA0320069096E0B8F1120F7DD158
:1075200014F8010B05900598EA2806D058A107A881
:1075300006F0CCFA0420069086E000F01FF9D6F899
:107540000D0034909DF8D3009DF8D210CDE90010C5
:107550009DF8D1309DF8D02050A125A806F0B6FAAC
:10756000012225A9002004F005FF4FF0000B0025A3
:1075700008E034A8405D18B90BF1010000F0FF0BE2
:10758000681C85B2042DF4DBBBF1020F07DB01227E
:1075900047A1002004F0EEFE0520069054E09DF87F
:1075A000D3009DF8D210CDE900109DF8D1309DF8A0
:1075B000D02041A125A806F089FA042234A9414827
:1075C000FCF7D1FE002838D000F0FEF8042234A9E0
:1075D0003C48FCF7C8FE04F085FA3A4886303A4940
:1075E000D1F81D10A0F19602D27CA0F196039B7CED
:1075F000CDE90032CDE902109638437C027C33A1FC
:1076000025A806F063FA07A925A8FDF701FE37A013
:1076100001F012FE07A801F00FFE00E023E037A002
:1076200001F00AFE012236A1002004F0A3FE64202E
:10763000DFF8D8C000DF00BFFEE735A107A806F0DD
:1076400045FA0020069000BF012207A9002004F09F
:1076500091FE3148007810B9012000F067F802204F
:107660002E49087000E000BF00BF16E71C01002093
:107670004C656E206572720053756D2065727200E4
:107680005479706520756E537570706F7274000058
:107690005269676874206572720000004E65774910
:1076A000503A25642E25642E25642E2564000000A2
:1076B0006572725F4950000025642E25642E256492
:1076C0002E256400F01800204C18002069703D251C
:1076D000642E25642E25642E25643B69643D256C4B
:1076E000753B7077643D25733B00000041542B507F
:1076F0004F433D3031303030300000000D0A000083
:107700005265626F6F742E2E2E000000E5EE0008A9
:1077100053616D655F495000D82700201601002095
:1077200001200149087070471C01002010B5044673
:1077300001200B49087000200A490880012C03D160
:10774000B4200949088002E03C2007490880002055
:1077500006490870012206A104F00CFE10BD0000CD
:1077600017010020180100201A0100201601002036
:107770000D0A537461727420636E74007047704711
:1077800010B504460121C80203F0BEFB7D2003F0C2
:1077900073FC08B103F0F8FB45F2555000F028F8EF
:1077A000062000F019F8A0B200F01CF800F00CF868
:1077B00000F002F810BD00004CF6CC400149086012
:1077C00070470000003000404AF6AA2001490860D6
:1077D00070470000003000400149486070470000D9
:1077E00000300040014988607047000000300040D0
:1077F00001490860704700000030004009480078E7
:10780000FF2804DA07480078401C0649087006483B
:107810000078FF2804DA04480078401C0249087008
:10782000704700008C0000208D00002010B58448B7
:1078300000680E2803D08248006807282BD1012257
:1078400080A1002004F096FD002081490870814944
:10785000087381480078032803D100207E4908700E
:1078600015E0DFF8F8C100DF7D490968884201D9D9
:107870000A2405E0DFF8E4C100DF794909680C1A41
:10788000A0B2DFF8E0C100DF77A001F0D5FC002056
:1078900079490870D2E06A4800680D2870D1012249
:1078A00076A1002004F066FD7748007801280DD10C
:1078B000022076490870002275A1032001F01CF80F
:1078C00000207A4908707A49086010BD774800782E
:1078D00003284EDA7748007802280DD10020754938
:1078E0000870002274A1032001F006F8012275A19E
:1078F000002004F03FFD3CE05748007878B10020BC
:107900006C4908705449087000226BA1032000F0F4
:10791000F3FF01226FA1002004F02CFD29E0714843
:10792000007888B94B48007800B9CEE700226EA1F4
:10793000032000F0E1FF012270A1002004F01AFDF5
:1079400001206849087014E066480078012803D0D7
:107950006448007802280CD1002062490870002297
:107960006AA1012000F0C8FF01226BA1002004F0F1
:1079700001FD00204D4908704D4908605EE0FFE7B9
:107980002F4800680B2859D1012267A1002004F07C
:10799000F1FC3D480078012810D13C4800780128CE
:1079A00002D105F073FE08E038480078022802D1C1
:1079B00005F06EFE01E003F0F9FC86E75D48006823
:1079C00002280EDD3048007858B95B48007800285E
:1079D00007DDFEF79FFB00205849087055490860F5
:1079E00073E75448006810F1020F0ADA5348007830
:1079F000032806D051480078092802D003F0AAFDD8
:107A000017E04E480078032813DA1248007801285E
:107A10000DD1104890F8260018B10E4890F8770064
:107A200010B903F0C3FC04E003F082FE01E003F0B0
:107A3000BDFC0020414908703E49086000BF44E792
:107A4000A40000205B50505420467265655D000024
:107A500090000020D82700203500002071F5000894
:107A60006C000020E5EE000841542B504F433D30A0
:107A700043303030300D0A008F0000205B4B4559F9
:107A80003120467265655D0005000020320000204F
:107A9000343735334137374546393542423238423B
:107AA00034383732324336370000000036000020C9
:107AB0003800002028000020303039304641353170
:107AC000000000005B457869744E657453656C5D19
:107AD000000000005B457869745573657253656CEE
:107AE0005D00000034000020413437464334374500
:107AF0003039393045393632000000005B456E744C
:107B0000657247726F757053656C5D004344434204
:107B100042334636000000005B4578697447726F57
:107B2000757053656C5D00005B4B455932204672A1
:107B300065655D003C000020F80000203700002053
:107B400008B50121084603F0FFF901211548FEF7A9
:107B500013FD01211C2003F0F7F948208DF80300E4
:107B600003208DF802004FF48050ADF80000694604
:107B70000D48FEF777FC4FF40040ADF80000694671
:107B80000948FEF76FFC0820ADF800006946074879
:107B9000FEF768FC0020064908703A210E2003F029
:107BA00031FF08BD0002300000080140000C014018
:107BB0008F00002000B589B078480068072806D0FB
:107BC0000B287DD00D2869D00E2866D100BF01207A
:107BD0007349087073490870012273A1002004F0F2
:107BE000C9FB7448007802281DD100207249087032
:107BF00001207249087000206E4908700120704908
:107C00000860704A70A101A805F060FF01A801F0AA
:107C100013FB012271A1002004F0ACFB1420DFF85B
:107C2000CCC100DF39E07248007802281ED1032061
:107C30006F4908706F48008A28B900226EA10120A0
:107C400000F05AFE0CE00A20DFF8A0C100DF5D4A18
:107C5000093A71A101A805F039FF01A801F0ECFA79
:107C6000012272A1002004F085FB16E07348007821
:107C7000022806D101207249087000206F4908705F
:107C80000BE0DFF8C0C100DF1E306F490860012043
:107C9000584908736DA001F0CFFA7BE000204149FC
:107CA000087001226DA104F065FB70480078072878
:107CB00051DA6E480078401C6C490870084600E0B4
:107CC0004AE00078032833D13A48007800282FD1C1
:107CD0004848007808B909B000BD0120444908703F
:107CE000012263A1002004F045FB002264A10120D1
:107CF00000F002FE0220DFF8F4C000DF65A001F012
:107D00009BFA0220DFF8E4C000DF00203949088236
:107D1000488201F11D0264A101A805F0D7FE0022EE
:107D200001A9012004F026FB01A801F085FA12E068
:107D30004E48007807280ED11E48007858B9002018
:107D40002B49087001225DA104F014FB02203B497D
:107D50000870FDF797FC1DE0002012490870012211
:107D60005AA104F007FB5D480078092811DA5B4846
:107D70000078401C5949087008460078032802D151
:107D800003F0EEFC05E055480078092801D103F026
:107D9000A9FD00BF00BF00BF9DE70000A4000020B8
:107DA000900000208F0000205B50505420507265DE
:107DB00073735D0034000020440000204200002066
:107DC000140C0140FA28002041542B504F433D3001
:107DD000393030303025730D0A0000005B4578697A
:107DE0007447726F757053656C5D0000E5EE0008B6
:107DF00035000020D827002043454445433645340C
:107E0000434246434233433944344231443444418B
:107E1000434644460000000041542B504F433D3040
:107E2000413030303025730D0A0000005B45786921
:107E3000745573657253656C5D0000002800002066
:107E40002900002071F500086C00002041542B50DF
:107E50004F433D3042303030300D0A005B4B4559C6
:107E6000312050726573735D000000003600002001
:107E70005B456E7465725573657253656C5D000089
:107E80004233433944344231443141314434463140
:107E90000000000041542B504F433D313030303012
:107EA0003032300D0A00000041542B504F433D301A
:107EB000453030303025730D0A0000005B456E748C
:107EC00065724E657453656C5D0000005B4B4559EF
:107ED000322050726573735D00000000370000208F
:107EE00000200E49096811F4805F01D040F00100C4
:107EF0000A49096811F4004F01D040F00200084916
:107F0000096811F0080F01D040F004000349096826
:107F100011F4006F01D040F00800704708080140DC
:107F2000080C014008B50121084603F00DF80121B5
:107F30001048FEF721FB01211C2003F005F810205A
:107F40008DF8030003208DF802001020ADF800002A
:107F500069460948FEF786FA4020ADF800006946F8
:107F60000548FEF77FFA10200349103108604020D1
:107F7000086008BD00023000000C014010B5044646
:107F800091210C2003F03EFDFCB1002068490870EF
:107F9000684908706849087068490870FF20684996
:107FA00008706849087000206749087067490870C0
:107FB00067490870FF2067490870674908701020FA
:107FC000664908604020086010BD59480078401C90
:107FD000C0B257490870092802DD0020087000E08F
:107FE000F2E75F48007818B910205C49086048E063
:107FF0005C48007820B910205849091F086040E00B
:108000004F48007856490978884205D14D48007894
:1080100054490978884219D00020464908704A49D5
:1080200008704F480078464908704E480078454926
:1080300008704B4800784006000E404908704148DF
:108040000078097801EB40003B4908703948007816
:10805000401CC0B23749087037490978884202DDB0
:108060000020344908703348007834490978884240
:1080700004DA10203949091F086002E0102037494E
:1080800008603948007818B940203449086048E051
:108090003648007820B940203049091F086040E088
:1080A0002C48007830490978884205D12A48007860
:1080B0002E490978884219D000201E4908702249AB
:1080C0000870294800782349087028480078224918
:1080D0000870254800784006000E1D4908701E48AB
:1080E0000078097801EB40001849087016480078BC
:1080F000401CC0B21449087014490978884202DD56
:108100000020114908701048007811490978884208
:1081100004DA40201149091F086002E040200F499D
:108120000860CF210C2003F06DFC00BF4CE700007D
:1081300078000020790000207A0000207B000020D9
:108140007C0000207D0000207E0000207F000020B9
:10815000800000208100002082000020140C0140DB
:1081600074000020750000207600002077000020B9
:108170001FB51948007800B91FBD18A001F05CF8C0
:108180001E20DFF868C000DF012019494872194934
:1081900008601148427818A1684605F097FC6846C7
:1081A00001F04AF80C48D0F8660020B90A48801C53
:1081B00001F042F804E00849D1F8660001F03CF80B
:1081C00011A001F039F80020034908701E20DFF8E3
:1081D0001CC000DF00BFCFE72839002041542B4CE2
:1081E00053485454535354500D0A0000E5EE000810
:1081F000D8270020140C014041542B4C53485454B0
:10820000533D25642C220000220D0A0070B586B073
:1082100005460E46144623462A4608A101A805F045
:1082200055FC01A801F008F82146304601F00FF88E
:1082300007A001F001F806B070BD000041542B54B6
:10824000435053454E443D25642C25642C000000CA
:108250000D0A000070B504460D4616463246294602
:108260002046FFF7D3FF3146284602F00FFE012CCF
:1082700008D109480078FF2804DA07480078401C34
:1082800005490870012C06D10448807820F00200CE
:10829000801C0249887070BD02000020B01D0020C3
:1082A0002DE9F04F93B0044689466178A07861F3D8
:1082B0001F208346012002905A467BA106A805F0A4
:1082C00005FC012206A9002004F054F8ABF570600B
:1082D00003387CD0A0F5E040FE387BD0FF2804D0E6
:1082E000A0F50070FF3874D14BE0E67B324671A1F7
:1082F00006A805F0EBFB012206A9002004F03AF8DD
:10830000052E2AD2DFE806F003151A1F24000027E5
:1083100006E007F11000215C6948C155781CC7B21E
:10832000072FF6DB03F0DEFB66A103A805F0CEFB0A
:1083300018E065A103A805F0C9FB13E065A103A837
:1083400005F0C4FB0EE065A103A805F0BFFB09E042
:1083500066A103A805F0BAFB04E067A103A805F035
:10836000B5FB00BF00BF03AB324665A106A805F010
:10837000ADFB012206A9002003F0FCFFFDF7F4F895
:1083800089E0E5784FF6FF7000EA052505F47F45A2
:1083900020790543681E85B2B5F5CA7F01DB4FF42D
:1083A000CA7540F295115A48FBF7A1FF2A4604F11D
:1083B0000E015748FBF782FF5548401EA0F8965122
:1083C000B0F89601002801DD03F0FAFD63E051E00A
:1083D00000E05DE00FFA89F8A8F10300215C401C81
:1083E00014F800A061F31F2A401C265C53464A463D
:1083F00048A106A8009605F069FB012206A9002005
:1084000003F0B8FFBAF1020F2CD0BAF5817F03D088
:10841000BAF5007F2CD11FE076B94648807820F06D
:10842000080008304349887043A106A805F04EFBB8
:108430003C204049887109E03E48807820F00800DF
:108440003C4988703EA106A805F040FB012206A920
:10845000002003F08FFF0BE001223CA1002003F07D
:1084600089FF05E001223DA1002003F083FF00BF4A
:1084700000BF10E0607B1249193981F8A600084658
:1084800090F8A61039A005F0FDFA03F02BFB02E0EE
:108490000020029000BF00BF029810B100203F49A9
:1084A000087013B0BDE8F08F0D0A636D643D253090
:1084B00034780000726573756C743D253032780035
:1084C000F91800204F6B00004361722045786973F2
:1084D000740000004E6F206361720000446576698D
:1084E0006365204578697374000000004E6F205268
:1084F00065636F72640000004661696C650000008E
:108500005B52656769737465725D2564202573002D
:10851000253500204C656E3D25642C61636B436DF1
:10852000643D253034782C726573756C743D25304C
:1085300032780000B01D00205B4154485D4F6B0055
:108540005B4154485D4661696C6500004C6F636136
:1085500074696F6E2041434B0000000048656172F2
:108560005469636B2041434B000000007375744EE7
:1085700065775365676D656E74506172612E5365E2
:108580006E6447707354696D653D3D3D3D3D3D3DB5
:108590003D3D3D3D3D3D25640D0A000002000020AB
:1085A00008B54FF4A06001F06FFA1D21012003F01F
:1085B00029FA25208DF8000001208DF801008DF8A2
:1085C00002008DF80300684601F024FA24210120FE
:1085D00003F018FA26208DF8000001208DF8010024
:1085E0008DF802008DF80300684601F013FA2B2184
:1085F000012003F007FA27208DF8000001208DF8F4
:1086000001008DF802008DF80300684601F002FABF
:108610003221012003F0F6F901208DF801008DF8D8
:1086200002008DF8030007208DF80000684601F075
:10863000F1F908208DF80000684601F0EBF91720E9
:108640008DF80000684601F0E5F908BD002640F20B
:10865000F231082003F0D6F9DFF87CC100DF5F4972
:1086600008604FF49A715E48FBF741FE01205D49B6
:10867000086064214FF45E7003F046FC0120594904
:10868000091F086002F02EFD5748B0F82F2000F1B6
:10869000210156A005F0F6F95348D0F81D1058A056
:1086A00005F0F0F9002059490870012258A103F0A3
:1086B00061FEFFF737FC01225AA1002003F05AFEA9
:1086C00000205B49086003F003FA0023594A5A4925
:1086D0005A48DFF86CC100DF5A49086000235A4A43
:1086E00055495A48DFF858C100DF5949086000234E
:1086F000584A48F203015848DFF844C100DF57499F
:10870000086040F20C41082003F07CF962E002F0BE
:108710002BFB0120DFF848C100DF40F215410820A3
:1087200003F070F94F48008828B14F4801F032FA41
:1087300000204C49088040F21B41082003F062F9F8
:10874000FEF716F9050006D0012D02D1FFF732FA27
:1087500001E0FFF76BF840F22641082003F052F9E0
:10876000FDF75EFB4148007803F0E4F90020FFF7D5
:1087700005FCDFF8FCC000DF3E490968884200D2F2
:1087800028E0DFF8ECC000DF64303A49086040F2CE
:108790003341082003F036F9FFF730F840F2354155
:1087A000082003F02FF9FEF7D7FA0446002C01DD6C
:1087B00031480460032E02DA701CC6B203E02E4872
:1087C0000068FDF705F9FDF79DFD05F0DDFFFDF7FC
:1087D0004BF800BF9BE700000DF8000824000020C4
:1087E000D8270020140C01404C1800200D0A2573D6
:1087F0005F5625642053746172742E2E2E0D0A006C
:1088000050534E3A256C750D0A00000032000020CE
:108810004D61696E205461736B20537461727421D1
:10882000000000004C656420496E6974206F6B0085
:108830003C0000201031002003000400B99700081C
:108840000DF60008F4000020102D0020859300088C
:10885000F0000020A8380020A5C90008340100203D
:10886000E5EE00080C000020CC0900206900002083
:1088700071F50008540000202C00002010B5124CA7
:1088800010212046FBF733FD10484069000E207090
:108890000E484069000C60700C48808A000AA07085
:1088A0000A48007DE07009480069000E2071074801
:1088B0000069000C60710548008A000AA071034835
:1088C000007CE07110BD000094380020B01D002035
:1088D00070B50546002407E0285D0D2802D1002070
:1088E000285570BD601C84B22846FBF735FDA042B8
:1088F000F2D800BFF5E700002DE9F04106460D462D
:1089000017462846FBF728FD84B2642C00DD64245A
:108910007FB9224629461048FBF7D0FC642C02DAC6
:1089200000210D48015500200B49891EC1F8660041
:1089300003E00948801EC0F866500748801E467054
:108940000078401C0449891E08700448DFF810C0F4
:1089500000DFBDE8F08100002A3900203801002046
:1089600015F30008044802680448018804A005F0D3
:1089700089F800BFFEE70000480000204600002004
:108980000D0A5B4D4D485D463D25642C4C3D2564EC
:108990000000000018B10221034A116003E0022127
:1089A000014A121F116070471408014008B50220E7
:1089B000ADF8000010208DF8030003208DF80200B0
:1089C00069460548FDF74EFD0120FFF7E3FFA021B2
:1089D000072003F017F808BD0008014010B59AB051
:1089E0002A4C2BA10BA805F071F82D4890F87400C3
:1089F00020B92CA10BA8FBF785FC12E0284A7432A1
:108A00002CA101A805F062F801A800F015FC244A89
:108A100074322EA101A805F059F801A90BA8FBF7A3
:108A200071FC00220BA9104603F0A4FC28A10BA89E
:108A300005F04CF81A4890F8540018B1184890F80E
:108A4000640020B917A10BA8FBF75CFC16E0144BDF
:108A50006433A3F1100221A101A805F037F801A8A1
:108A600000F0EAFB0E4B6433A3F1100221A101A830
:108A700005F02CF801A90BA8FBF744FC01220BA977
:108A8000002003F077FC1AB010BD0000B6050020EE
:108A90005B31315D416363657373703A00000000C0
:108AA0004C180020756E737570706F72742D456D63
:108AB0007074790041542B4D495050524F46494CE7
:108AC000453D312C222573220D0A0000257300003C
:108AD0002C4E616D652D506173733A0041545E50A8
:108AE00050504346473D222573222C222573220DE8
:108AF0000A00000025732C2573000000F0B5BDB0FE
:108B0000384C40F28B11022002F07CFF002664E01A
:108B100035A000F091FB32275AE040F21441A01C2E
:108B200000F082FE208000284ED033A1A01C00F06F
:108B300015FC00284CD13248D0F81D2031A12EA8B8
:108B400004F0C4FF3148C07C3049897CCDE9001075
:108B50002E48437C027C2EA103A804F0B7FF03A992
:108B60002EA8FBF7CFFB294A96322DA103A804F0CB
:108B7000ADFF03A92EA8FBF7C5FB0DA92EA8FCF796
:108B800047FB002507E0A01C405D0D2802D1002115
:108B9000A01C41556D1CA01CFBF7DEFBA842F2D8BF
:108BA0000DA904F10F00FBF7F4FB58B11EA000F073
:108BB00043FB0DA800F040FB1FA000F03DFB01208F
:108BC0003DB0F0BD0020FBE70120DFF870C000DF02
:108BD0003800A7F10107A0D1761C052E98DB0020F4
:108BE000EEE70000B605002041542B504F433D30C6
:108BF00032303030300D0A002B504F433A303200C3
:108C00004C18002069643D256C753B00E01800207D
:108C100069703D25642E25642E25642E25643B0055
:108C20007077643D25733B0041542B504F433D30DA
:108C300031303030300000000D0A0000E5EE000851
:108C40002DE9FE430025224C4FF40971022002F069
:108C5000D9FEA846002636E0322745B901251DA0D9
:108C600000F0EAFA1EA1684604F030FF07E0002594
:108C70001DA000F0E1FA1FA1684604F027FF1CE0E8
:108C800040F21441A01C00F0CFFD208088B169465D
:108C9000A01C00F063FB80B9E81DA11C085C5228F1
:108CA0000BD105F10900085C412806D10120BDE87F
:108CB000FE830120DFF844C000DF3800A7F1010186
:108CC000CFB2DDD1761C1E2EC6DB0020EFE7000000
:108CD000B605002041542B514350494E3F0D0A0028
:108CE0002B514350494E3A0041542B4350494E3F7B
:108CF0000D0A00002B4350494E3A0000E5EE0008F3
:108D0000F0B595B03B4C002700256AE064263AA0F8
:108D100000F092FA60E040F21441A01C00F084FDE3
:108D20002080002854D037A1A01C00F017FB002899
:108D300052D1142204F109013448FBF7BFFA334A37
:108D400033A101A804F0C2FE304800798DF800007C
:108D50002E4840798DF8010000208DF80200684609
:108D6000FBF728FC0C2825D2DFE800F00F061019CD
:108D700024241A111B07241C00BF02202849087054
:108D800028A101A8FBF7BEFA19E000BF00BF01202F
:108D90002349087027A101A8FBF7B4FA0FE000BF30
:108DA00000BF00BF00201E49087026A101A8FBF7E4
:108DB000A9FA04E027A101A8FBF7A4FA00BF00BFAD
:108DC000012201A9002003F0D5FA012015B0F0BD61
:108DD0000120DFF890C000DF3000A6F101069AD133
:108DE0006D1C052D92DB01221FA1002003F0C2FAA9
:108DF0000020EBE7B605002041542B49434349448A
:108E00000D0A00005E534349443A0000103500202B
:108E10005B30395D49434349443A25735B000000A8
:108E2000F90000204348494E415F554E49434F4D9C
:108E30005D0000004348494E415F4D4F42494C455B
:108E40005D0000004348494E415F54454C45434F47
:108E50004D5D0000554E4B4E4F572D4943434944FD
:108E60005D000000E5EE00085B30395D4765742069
:108E700043434944206661696C6564002DE9F0470D
:108E80008CB05D4C4FF4DA71022002F0BBFD4FF064
:108E9000000A012259A1002003F06CFA0026B04616
:108EA000A3E01EB959A000F0C7F902E059A000F0F4
:108EB000C3F94FF032098FE040F21441A01C00F0DA
:108EC000B3FC208000287DD0C6B955A1A01C00F0BD
:108ED00045FA28B90022A11C104603F04BFA7BE0AA
:108EE00053A1A01C00F03AFA002875D10022A11C61
:108EF000104603F03FFA701CC6B273E04EA1A01CEE
:108F000000F02CFA28B90022A11C104603F032FA16
:108F100062E04EA1A01C00F021FA38B90022A11C89
:108F2000104603F027FA0CB0BDE8F08748A1A01C5A
:108F300000F014FA00284FD10022A11C104603F0C3
:108F400019FA002700253BE0A01C405D5F2836D1C0
:108F5000781CC7B2012F0AD1A01CE91C405C8DF817
:108F60000400A01C291D405C8DF8050027E0032F9C
:108F700025D1A01CA91C405C8DF80600A01CE91C92
:108F8000405C8DF80700A01C291D405C8DF808008E
:108F9000A01C691D405C8DF8090000208DF80A00B6
:108FA00001AA2FA104A804F091FD012204A9002028
:108FB00003F0E0F901A8FBF7FDFA2D4908606D1CEC
:108FC000A01C00E004E0FBF7C7F9A84204D9BBE706
:108FD0000120DFF8A0C000DF5FEA0900A9F1010964
:108FE0007FF46AAF00BF08F10108B8F10A0FFFF67D
:108FF00058AF00BF97E70000B60500205B30335D37
:109000004D6F64656D496E666F3A00004154490DBD
:109010000A00000041542B4C435453570D0A0000E2
:109020004D616E7566616374757265723A00000019
:109030004D6F64656C3A0000536F667477617265BA
:1090400056657273696F6E3A0000000041503A0035
:10905000496E6E657256657273696F6E3A000000F4
:109060005B30335D4D6F64656D5665723A257300F4
:10907000B4000020E5EE000808B500F0BFFC1020A9
:109080008DF8030003208DF802004FF48050ADF8F6
:10909000000069461B48FDF7E5F94FF40050ADF8B4
:1090A000000069461748FDF7DDF94F21022002F064
:1090B000A9FC0020144908705321022002F0A2FCF0
:1090C0004FF480500F49103108606420DFF83CC035
:1090D00000DF4FF480500B49143108604000091F35
:1090E00008606420DFF824C000DF4FF40050054919
:1090F0001431086004F0E2FB08B1002008BD012033
:10910000FCE70000000C014002000020E5EE000832
:109110002DE9F0438BB0354C002559E04FF0320972
:1091200033A000F089F84AE040F21441A01C00F09E
:109130007BFB208000283ED031A1A01C00F00EF95E
:1091400000283CD1A01CFBF707F907B24FF000083C
:1091500000252DE0A01C405D0D2817D1002001A99D
:1091600001F8080001A8FBF725FA06B2A31C324655
:1091700026A101A804F0AAFC002201A9104603F0D0
:10918000F9F8274806600BB0BDE8F083A01C405DED
:1091900030280BDBA01C405D392807DCA01C425D99
:1091A0004046411C0FFA81F801A90A54681C05B217
:1091B000BD4204DACEE70120DFF868C000DF5FEAD5
:1091C0000900A9F101010FFA81F9ADD1681C05B2BE
:1091D000052DA3DB324614A101A804F077FC01227F
:1091E00001A9002003F0C6F800BFCCE7B6050020B7
:1091F00041542B504F435F5645523F0D0A0000002B
:109200002B504F435F5645523A0000005B30345DAF
:10921000504F437665723A25643C2D3E257300001D
:10922000B8000020E5EE00085B30345D506F6356F7
:1092300065723D256400000070B504462046FBF7CA
:109240008BF805462946204604F0BAF970BD70B582
:1092500004460D462946204604F0B2F970BD0000D0
:109260002DE9F041204C002635E0322700BF1FA039
:10927000FFF7E2FF28E040F21441A01C00F0D4FA0E
:10928000208000281CD01EA1A01C00F067F8D8B9CF
:1092900004F10F00FBF78EF90546A5F5D8505838B4
:1092A00007D01BA0FFF7C8FF0120DFF880C000DF58
:1092B000DDE701221EA1002003F05CF8BDE8F0818B
:1092C0000120DFF868C000DF3800A7F10101CFB24C
:1092D000D1D1701CC6B2052EC7DB012219A1002016
:1092E00003F048F800BFE9E7B605002041542B4CD5
:1092F000534854545353504545443F0D0A00000011
:109300002B4C534854545353504545443A000000A5
:1093100041542B4C534854545353504545443D2DD0
:10932000312C373030300D0A00000000E5EE000827
:109330005B30365D536574545453205370656564D7
:10934000204F6B005B30365D53657454545320538B
:1093500070656564204661696C65640030B50246DD
:109360000B461946144607E008782578A84201D034
:10937000012030BD491C641C08780028F4D100BFCE
:10938000F7E700008AB00025B64C0120B649087006
:109390000122B6A1002002F0EDFF0120FDF7A8FE9A
:1093A0000020B649087003F047F90020B44948701E
:1093B0008870C870B34BB4A22821684604F072FBD1
:1093C00001226946002002F0D5FF0122B2A100204F
:1093D00002F0D0FF0122B5A1002002F0CBFF00BFB8
:1093E0000020B64908702020B5490860012002F02D
:1093F00041FE4FF49A71B348FAF779FFFFF73CFE4C
:1094000028B101226946002002F0B4FF13E02020B9
:10941000AB49091D08600122ABA1002002F0AAFFA0
:10942000FCF778FE06E00020A64988736420DFF888
:10943000B4C200DFF7E74FF40071A1481038FDF720
:10944000E3F8012802D1A849087003E020209C49D4
:10945000091D0860012099490870A4A0FFF7ECFEDF
:109460000122A4A1002002F085FFFFF707FDFFF70E
:109470004FFEFFF7F5FE04F0ABF9FFF7E1FB002824
:1094800039D140F6AC55FDF7E1F833E040F2144134
:10949000A01C00F0C9F9208000B12BE00120DFF80A
:1094A00044C200DF96480088002805DD954805F095
:1094B0001FFC0020924908800020824988736A4876
:1094C000007800B916E0681C80B20546B0F57A7FD6
:1094D00001DB002500E00DE000228BA10320FFF757
:1094E0000BFA01207649086001228BA1002002F0CE
:1094F00041FF00BFCAE701228CA1002002F03AFF21
:10950000FFF7FEFBFFF7FAFA28B101228BA100203A
:1095100002F030FF04E001228CA1002002F02AFFBB
:10952000FFF75CFA01228DA1002002F023FFFEF775
:10953000F7F8FDF78BF801206249C87201228CA16F
:10954000002002F017FF8BE047480078C8B940F2CE
:109550001441A01C00F068F9208068B10022A11C11
:10956000104602F007FF86A1A01CFFF7F7FE38B9EE
:10957000052002F07FFD03E00120DFF868C100DF75
:109580006EE040F21441A01C00F04EF92080C8B1FA
:10959000A0782B2802D0A078242808D1002049499F
:1095A00088730022A11C104602F0E4FE00E057E0A0
:1095B000A01C01F09BF8012800D151E0A01CFBF792
:1095C00081FE4DE00120DFF81CC100DF3D4800783E
:1095D00018B9012002F04EFD16E03A48007A002842
:1095E00003DD032002F046FD0EE03648807A0028B5
:1095F00007DD3448007B002803DD042002F03AFD3B
:1096000002E0022002F036FD0020FDF771FD1C484B
:109610004078012801D1FEF7B2F802F01BFA04F0FD
:10962000A5F9284890F8300100B1D9E6DFF85CC10F
:1096300000DF57490968884200D211E0DFF84CC1C9
:1096400000DF00F596705249086052A0FFF7F4FD64
:109650000120DFF890C000DF52A0FFF7EDFD00BF52
:1096600072E70000B6050020F8000020506F63206C
:109670005461736B207374617274210002000020C6
:10968000EB000020761900205B30315D6861726468
:1096900049443A25730000004D6F64656D205461A4
:1096A000736B207374617274210000004D6F6465E8
:1096B0006D496E69742E2E2E0000000030000020CF
:1096C000100C0140D82700205B30315D4661696C89
:1096D00065640D0A456E746572204754204D6F64B1
:1096E00065210000E5EE00083100002041544530BE
:1096F0000D0A00005B30325D41544530204F4B0075
:109700001A000020A80E0020463738424432363373
:1097100036313533000000005B30385D4E6F205528
:10972000494D204361726421000000005B30385DC8
:109730004361726420726561647900005B31305D61
:109740005273745F504F4350617261005B31305D02
:10975000504F43207374696C6C0000005B31325DC4
:109760004869676F73536572496E69740000000041
:109770004D6F64656D4C6F6F70537461727400004F
:109780005E4D53473A5175697400000071F5000849
:10979000FC00002041542B4D4F444F445245583F4C
:1097A0000D0A000041542B4C43544D4F424150523E
:1097B00045463F0D0A00000000210748DFF81CC0A5
:1097C00000DF07E04FF6FF710348DFF814C000DF49
:1097D00003F002FDF6E7000004010020D5F20008C6
:1097E0004DF30008202009490860012208A100204B
:1097F00002F0C0FDFCF78EFC06E0002008498873EB
:109800006420DFF820C000DFF7E70000140C0140FF
:10981000676F2047545F4D6F64650D0A00000000BC
:10982000D8270020E5EE00082DE9F84380460E46D3
:10983000314C3248007820B931A004F023F9FFF709
:10984000D1FFA08810B90020BDE8F8836188A01D71
:1098500030F82100ADF800006188A01D00EB810008
:109860004088ADF802000027002524E0B4F8D000BD
:1098700000B924E004F1CE04D4F80A00E18810F81D
:109880000190E08800F10100E080E08834F8CE1912
:10989000884202DB0020A4F8D400B4F8D000401EB7
:1098A000A4F8D000B74204DA3846791C8FB208F821
:1098B0000090681C85B2BDF80000A842D6DC00BF4D
:1098C0006088401C60806088322801DB0020608056
:1098D000A088401EA080BDF80000A84201D0FE2054
:1098E000B2E7BDF80000B04201DDFF20ACE7BDF8F3
:1098F0000000C0B2A8E7000070170020F8000020A8
:1099000053544F5020474F2047540D0A0000000089
:1099100030B503460A4613480024048084804480FE
:10992000002108E00025841D04EB81046580841D6E
:1099300024F82150491C3229F4DBC0F8D83000212A
:1099400004E00024D0F8D8506C54491C9142F8DB54
:1099500020F8CE2F00248480C4804480A0F1CE0063
:1099600030BD00007017002070B504460A46224939
:109970008888322801DBFF2070BDB1F8D000104488
:10998000B1F8CE50A84201DDFE20F5E7B1F8D25083
:109990000E88881D00EB860045800D88881D20F804
:1099A0002520002319E0E05C01F1D201D1F8065036
:1099B0000E88A855088800F10100088031F8D20906
:1099C000B0F5006F02DB0020A1F8D200B1F8D000A2
:1099D000401CA1F8D000581C83B29342E3DB0888F6
:1099E000401C08800888322801DB00200880888815
:1099F000401C88800020BFE77017002000B54FF49E
:109A000000610248FFF784FF00BD0000700F0020D6
:109A10007047000070B5002100230F22C4780CB3FA
:109A2000164C246804F4E064C4F5E064210AC1F132
:109A30000403CA40447804FA03F1847814402143B3
:109A400009010F4C0678A155047804F01F05012484
:109A5000AC4005786D114FF0E02606EB8505C5F8A2
:109A6000004109E0047804F01F050124AC40054DD5
:109A70000678761145F8264070BD00000CED00E038
:109A800000E400E080E100E002490143024A116085
:109A9000704700000000FA050CED00E02DE9F041F0
:109AA00007460C463846FAF757FC80460025002644
:109AB00022E0332228466D1C2254BA5D28466D1CD4
:109AC0002254302228466D1C225428466D1C2254F4
:109AD000A8F10100B04200D110E0322228466D1CEE
:109AE0002254302228466D1C225428466D1C2254D4
:109AF00028466D1C2254761C4645DADB00BF002048
:109B00006055BDE8F08100000B48016801F4007069
:109B1000B0F5007F0BD109480078052805DA074821
:109B20000078401C054A107004E0012070470020B6
:109B3000024A10700020F9E7080C01404C00002098
:109B40000EB50121084601F0FFF904208DF803004D
:109B500003208DF802004FF40070ADF80000694654
:109B60000B48FCF77FFC09210120FCF75BFC4FF45C
:109B70000070019000208DF8080008208DF8090081
:109B800001208DF80A0001A8FCF7D2F80EBD0000F4
:109B9000000C01402DE9F04FADF5137D82465022B7
:109BA000FA497FA8FAF78AFB002700200690059063
:109BB000FD21082001F026FF00BF38467F1C7FA949
:109BC00051F8200000780028F7D17F1E4FF48071F3
:109BD000082001F017FF002621E07FA850F826900A
:109BE0000AF1030B0020079008900FE099F800009D
:109BF0009BF80010884202D0012007900AE009F18A
:109C000001090BF1010B0898401C089099F800001D
:109C10000028EBD100BF079800B902E0761CBE42D5
:109C2000DBDB00BF4FF48A71082001F0EBFEBE427F
:109C300003D10DF5137DBDE8F08F132E22D2DFE89E
:109C400016F0130022002E004F00E30035015501ED
:109C50007D018C019801BC02CA02F5020B032003AE
:109C600069037E03C803F103092002F03BFA0122D5
:109C7000C7A1002002F07EFB0220FBF7EDFE0120D1
:109C8000C6490860DAE3092002F02CFA0122C4A1D7
:109C9000002002F06FFB0120FBF7DEFECEE309207F
:109CA00002F020FA0122C1A1002002F063FB022091
:109CB000FBF7D2FE1020B94908604020091F086058
:109CC000C001086040100860091D086007E0FDF74A
:109CD0007BFDFFF719FF10B12020B0490860F6E7BF
:109CE00059AAB5A15046FCF729FF0446012C01DB17
:109CF000282C05DB0122B1A1002002F03BFB9DE3F3
:109D000059A909A8FAF73CFB59AAB2A15046FCF799
:109D100015FF04460CB900250BE0052C05DD0122DA
:109D2000AEA1002002F026FB88E359A8FAF742FC16
:109D300085B259AAB0A15046FCF700FF0446012C99
:109D400001DB0A2C05DD0122ACA1002002F012FB90
:109D500074E359A8FAF73BFC8046AF48C0F81D8071
:109D60000120069009A9AD48FCF758FF28B101224F
:109D700092A1002002F0FEFA60E3A8481038858125
:109D800001200590A5488630FAF7E6FA0E2805D29C
:109D90000122A3A1002002F0EDFA4FE39F48863094
:109DA00000909D48D0F81D3009AAA4A159A803F03D
:109DB0008DFE0EA959A8FBF72BFAA6A0FFF73CFAD7
:109DC0000EA8FFF739FAA7A0FFF736FA9248D0F8A5
:109DD0001D00924910398989904A103AD27C8F4BE4
:109DE000103B9B7CCDE90032CDE902108B48103846
:109DF000437C027C9CA159A803F068FE012259A96A
:109E0000002002F0B7FA19E359AA6BA15046FCF7FB
:109E100095FE0446012C01DB282C05DB01229CA1C8
:109E2000002002F0A7FA09E359A909A8FAF7A8FA4D
:109E300059AA68A15046FCF781FE04460CB90025DA
:109E40000BE0052C05DD012297A1002002F092FA1B
:109E5000F4E259A8FAF7AEFB85B209A96F48001DD4
:109E6000FCF7DCFE28B1012289A1002002F082FA71
:109E7000E4E26A481038C58101200590674810382F
:109E8000C189C07D654A103A927DCDE900200291DA
:109E900062481038437D027D8AA159A803F016FE5E
:109EA000012259A9002002F065FAC7E25B48103888
:109EB000C07C5A491039897C584A103A527C574B19
:109EC000103B1B7CCDE90032CDE902105248D0F89E
:109ED0001D20524B86332D49A83159A803F0F6FDB9
:109EE000012259A9002002F045FAA7E2092002F058
:109EF000F9F801227BA1002002F03CFA0120DFF8F2
:109F0000F0C100DF0220FBF7A7FD4FF4005023490A
:109F100008604010091F08600520DFF8D4C100DF89
:109F20004FF480501D49086007E0FDF74DFCFFF736
:109F3000EBFD10B1202019490860F6E73648B0F86B
:109F40002F3000F121026BA159A803F0BFFD0122BF
:109F500059A9002002F00EFA70E26A486AA102686C
:109F600059A803F0B3FD012259A9002002F002FA1A
:109F700064E259AA68A15046FCF7E0FD0446002CB3
:109F800001DB0F2C01DD0122CAE0CEE090F80008D1
:109F900047542B544D3A4F4B00000000140C014025
:109FA00047542B54473A4F4B0000000047542B4472
:109FB0004D3A4F4B000000004950000047542B53CE
:109FC0004D503A4641494C5B495020496E76616C90
:109FD00069645D00506F72740000000047542B5399
:109FE0004D503A4641494C5B506F727420496E7631
:109FF000616C69645D00000050534E0047542B5360
:10A000004D503A4641494C5B50534E20496E766163
:10A010006C69645D000000004C180020F0180020FE
:10A0200047542B534D503A4641494C5B4D454944AA
:10A0300020496E76616C69645D00000069703D25A1
:10A04000733B69643D256C753B7077643D25733BBC
:10A050000000000041542B504F433D303130303030
:10A06000300000000D0A000047542B534D503A4970
:10A07000503D25642E25642E25642E25643B506FAB
:10A0800072743D25753B50534E3D256C75000000A4
:10A0900047542B5347503A4641494C5B495020495D
:10A0A0006E76616C69645D0047542B5347503A46A5
:10A0B00041494C5B506F727420496E76616C6964E3
:10A0C0005D00000047542B5347503A49503D2564EA
:10A0D0002E25642E25642E25643B506F72743D2519
:10A0E000753B000047542B5053543A4F4B0000002F
:10A0F000E5EE000847542B5645523A25735F562526
:10A10000640000002C00002047542B4241543A20A8
:10A1100025642056000000004163636F756E740073
:10A12000CEA1002002F026F983E524B90020D3490E
:10A1300081F8540004E059A9D0485430FAF720F9C6
:10A1400059AACFA15046FCF7F9FC0446002C01DBCC
:10A150000F2C05DD0122CDA1002002F00BF968E5EE
:10A1600024B90020C54981F8640004E059A9C34816
:10A170006430FAF705F901200690C04B6433A3F16F
:10A180001002CAA10EA803F0A1FC01220EA9002012
:10A1900002F0F0F8CDA0FFF74FF8B8485430FFF7C1
:10A1A0004BF8CDA0FFF748F8B4486430FFF744F807
:10A1B000AFF25010FFF740F840E1B04B6433A3F129
:10A1C0001002C6A10EA803F081FC01220EA90020F6
:10A1D00002F0D0F832E159AAC8A15046FCF7AEFC13
:10A1E000044624B159A8FAF7E5F9064601E040F221
:10A1F0006E3659AAC2A15046FCF7A0FC044624B111
:10A2000059A8FAF7D7F985B200E05025294630461B
:10A2100001F036FE2B463246BAA159A803F056FC8F
:10A22000012259A9002002F0A5F807E1B948C08928
:10A23000B849C97DB74A927DCDE900210290B54861
:10A24000437D027DB4A159A803F040FC012259A925
:10A25000002002F08FF8F1E0AE488188C078AD4A66
:10A260009278CDE900200291AA4843780278B2A101
:10A2700059A803F02BFC012259A9002002F07AF81A
:10A28000DCE059AAAFF2D0215046FCF757FC044657
:10A29000012C01DB282C05DB0122AFA1002002F0FC
:10A2A00069F8CBE059A909A8FAF76AF859AAAFF2F8
:10A2B000DC215046FCF742FC04460CB900250BE0BB
:10A2C000052C05DD0122ABA1002002F053F8B5E01A
:10A2D00059A8FAF76FF985B209A98E48FCF79EFCD8
:10A2E0008C488580012005908A4880888949C978F2
:10A2F000884A9278CDE90021029086484378027816
:10A30000A3A159A803F0E2FB012259A9002002F001
:10A3100031F893E07F484189407A7E4A127ACDE94C
:10A32000002002917B48C3798279A1A159A803F04A
:10A33000CDFB012259A9002002F01CF87EE059AAA9
:10A34000AFF28C315046FCF7F9FB0446012C01DBDF
:10A35000282C05DB01229EA1002002F00BF86DE005
:10A3600059A909A8FAF70CF859AAAFF29831504642
:10A37000FCF7E4FB04460CB900250BE0052C05DDD9
:10A3800001229AA1002001F0F5FF57E059A8FAF741
:10A3900011F985B209A95F48801DFCF73FFC5D48B3
:10A3A0004581012005905B4840895A49497A594ABC
:10A3B000127ACDE9002102905648C379827992A1A0
:10A3C00059A803F083FB012259A9002001F0D2FF14
:10A3D00034E059AA94A15046FCF7B0FB0446002C87
:10A3E00001DB1E2C05DD012291A1002001F0C2FF3E
:10A3F0001FE424B90020214981F8740004E059A920
:10A400001E487430F9F7BCFF012006901B4A7432D5
:10A410008FA10EA803F05AFB01220EA9002001F023
:10A42000A9FF0BE0154A74328EA159A803F04EFB28
:10A43000012259A9002001F09DFF00BF00BF06982E
:10A4400008B101F063FB059808B101F04BFB4FF434
:10A450000971082001F0D6FA00BF65E647542B4188
:10A46000504E3A4641494C5B4163636F756E7420B0
:10A47000496E76616C69645D000000004C18002034
:10A4800050617373776F72640000000047542B4172
:10A49000504E3A4641494C5B50617373776F72641A
:10A4A00020496E76616C69645D00000047542B4161
:10A4B000504E3A4163636F756E743D25733B506136
:10A4C0007373776F72643D25733B000041542B5AC0
:10A4D0005049445057443D002C00000047542B5233
:10A4E00041504E3A4163636F756E743D25733B5026
:10A4F000617373776F72643D25733B004600000003
:10A5000054000000424545503D2564487A2C25649E
:10A510006D730000E018002047542B5247503A4911
:10A52000503D25642E25642E25642E25643B504F16
:10A5300052543D25643B000047542B524D49503A3C
:10A5400049503D25642E25642E25642E25643B50FC
:10A550004F52543D25643B0047542B534D49503ACC
:10A560004641494C5B495020496E76616C69645D97
:10A570000000000047542B534D49503A4641494C86
:10A580005B506F727420496E76616C69645D000087
:10A5900047542B534D49503A49503D25642E25646C
:10A5A0002E25642E25643B506F72743D25753B004B
:10A5B00047542B524349503A49503D25642E256457
:10A5C0002E25642E25643B504F52543D25643B009C
:10A5D00047542B534349503A4641494C5B4950201C
:10A5E000496E76616C69645D0000000047542B532E
:10A5F0004349503A4641494C5B506F727420496E52
:10A6000076616C69645D000047542B534349503AAE
:10A6100049503D25642E25642E25642E25643B502B
:10A620006F72743D25753B00416363657373700001
:10A6300047542B534143433A4641494C5B41636382
:10A640006573737020496E76616C69645D0000000B
:10A6500047542B534143433A416363657373703DE1
:10A6600025733B0047542B524143433A4163636592
:10A670007373703D25733B002DE9F0418EB00646A3
:10A680004FF000080025002700BF13E0745D302C58
:10A6900001DB332C00DD10E06D1C745D302C01DB20
:10A6A000332C00DD09E0332C01D1781C87B26D1CFE
:10A6B00008F10108B8F5967FE8DB00BF074807827C
:10A6C0003A4607A101A803F001FA012201A91046A8
:10A6D00001F050FE0EB0BDE8F0810000D827002048
:10A6E0005B4F4C557365723D25645D0070B59AB043
:10A6F000044660784C2817D1A078532814D1E0780C
:10A70000482811D1207954280ED1607A45280BD1E0
:10A710000020F84948720846007A10B90120F6492D
:10A72000086001201AB070BD607930283FD1A0794F
:10A7300042283CD1E079462824D1207A462821D1EC
:10A74000EC484068032810D9EA4890F82F0160B916
:10A75000E848407848B9E748807830B90022E7A156
:10A760000120FEF7C9F80020DCE70020E949087065
:10A770000120E149091D08600C214FF4936001F0AC
:10A780007FFB12E0E07930280FD1207A30280CD1FD
:10A790000120D8498872DF490870D749091D08602F
:10A7A0000C2140F26E3001F06BFB0120BAE76079BA
:10A7B000382871D1A07942286ED1E07930286BD148
:10A7C000207A31280ED10120CA4988720220D2494C
:10A7D00008600020C74908720120C7490860C549C0
:10A7E000087009E0207A302806D10020C14988721B
:10A7F0000220C949091F0860607A30281ED1A07A5A
:10A8000030281BD1C348007801280AD10020C14953
:10A810000870B848007A10B10020B64908720120CB
:10A8200080E70020B34908720120B349091D086080
:10A830000C2140F26E3001F023FB2AE0607A3028D0
:10A840000FD1A07A31280CD10120AA4908700872D2
:10A85000A949091D08600C2140F26E3001F010FB7F
:10A8600017E0607A312814D1A07A332811D1A94891
:10A870000078012802D10020A649087001209D49D6
:10A8800008729D49091D08600C214FF4936001F086
:10A89000F7FA012046E7FFE76079382879D1A079F7
:10A8A0003228FBD1E0798DF80400207A8DF805007C
:10A8B00000208DF8060001A8F9F77CFEC6B236B17B
:10A8C000012E67D0022E6FD0032E6ED1B8E08948DA
:10A8D000007810B10120FCF729FF0020854908709D
:10A8E0008E48807820F008008C4988708CA101A8DF
:10A8F00003F0ECF8607C42282CD1A07C352829D1CB
:10A90000607E432826D1A07E412823D10520864998
:10A9100008707848407860B98448007848B90022C7
:10A9200083A10120FDF7E8FF0120724981F82F0182
:10A930000BE0704890F82D013C2806DB00206D49A3
:10A9400081F82D01012081F82F0180A101A8F9F7DC
:10A95000D9FC41E0607C43283AD1A07C452837D11E
:10A96000607E432834D1A07E322831D161484078BE
:10A97000E0B9604890F82F0128BB6C48007810BB04
:10A980005C48807838B900225CA10120FDF7B4FF53
:10A9900019E05EE026E057488078012813D10022B4
:10A9A0006EA1FDF7A9FF0EE022E04FE0514890F8BC
:10A9B0002E013C2807DB4F4890F82F0118B90020E2
:10A9C0004C4981F82E016AA101A8F9F79BFC03E02C
:10A9D0006AA101A8F9F796FC012201A9002001F063
:10A9E000C9FC33E0012268A1002001F0C3FC2DE086
:10A9F00004F11100F9F7B0FC801EC5B2512D00DB47
:10AA000051252A4604F111013A482630F9F798FCFD
:10AA1000512D03DA0021374826304155002060745B
:10AA2000092204F1090133481430F9F789FC0122A5
:10AA300058A1002001F09EFC01205949087005E052
:10AA4000012258A1002001F095FC00BF00BF0120A9
:10AA500068E6607938284BD1A079362848D1FCF7D0
:10AA60008DFE0120234908701E202F490870207A8E
:10AA700030283BD104F11100F9F76EFC801EC5B2FD
:10AA8000512D00DB51252A4604F111011948773078
:10AA9000F9F756FC512D03DA00211648773041555D
:10AAA00000206074092204F1090112481D30F9F7F1
:10AAB00047FC10484078D0B93948007830B90D4A81
:10AAC00077323BA101A803F001F80AE000203449E5
:10AAD0000870084B7733A3F1510236A101A802F0A8
:10AAE000F5FF002201A90120FDF706FF83E06DE0DC
:10AAF00086E00000D8270020100C01404345444563
:10AB0000434446384332453743314143424444335A
:10AB100000000000BD00002014080140B01D00200E
:10AB20005B6D73675D000000430000206A00002039
:10AB30004435434142414335443043354346413235
:10AB40004234454443454633000000004C6F67697A
:10AB50006E206661696C65640000000043454445F1
:10AB600042374138433141434244443300000000FE
:10AB70004E6F206E6574776F726B00004E6F206CA5
:10AB80006F67696E000000006C6F67696E20696E08
:10AB9000670000006C6F67696E206F6B000000003B
:10ABA000BC0000206C6F676F757420696E670000D1
:10ABB0002573000025733243443244314235433714
:10ABC0004332424432432573000000004D48007870
:10ABD00001280DD100204B4908704B4A4BA101A818
:10ABE00002F074FF002201A90120FDF785FE02E0BA
:10ABF0004AA002F047FF012043497739487091E5A8
:10AC0000607938280AD1A079332807D1E079302833
:10AC100004D1207A302801D1012083E560793828D9
:10AC20000AD1A079332807D1E079302804D1207ADD
:10AC3000312801D1012075E56079392807D1A07943
:10AC4000312804D1E01DFFF717FD01206AE5607986
:10AC5000302804D1A079652801D1012062E560790E
:10AC600038280DD1A07934280AD12046FDF730FECE
:10AC7000002204F109010120FDF73EFE012051E50B
:10AC80006079322816D1A079312813D12046FDF7FA
:10AC90001FFE002204F115010120FDF72DFE00200A
:10ACA0006075092204F10D011748A230F9F748FB3D
:10ACB000012037E56079312821D1E07930281ED193
:10ACC000A07B372802D0A07B382818D10E48AB30A3
:10ACD0000021016041600172D4F813100160D4F8C2
:10ACE00017104160E17E01722046FDF7F1FD002260
:10ACF00004F11F010120FDF7FFFD012012E50020F6
:10AD000010E50000420000204F2800204244463851
:10AD100043384542324325730000000053657442B6
:10AD20006565702E2E2E2E2E2E2E2E2E2E2E2E2E93
:10AD30002E0D0A0008B501211C2000F005F9102095
:10AD40008DF8030003208DF802002020ADF80000EC
:10AD500069460448FBF786FB20200249143108604D
:10AD600008BD0000000C014000B589B036480078ED
:10AD700008B909B000BD4FF4804034490860012291
:10AD800033A1002001F0F6FA35A0FEF755FA1020A5
:10AD90002E49091D086006203549088049E0012038
:10ADA000344908700A203449087025E0304800888A
:10ADB00088B13048007838B940202449091D08601E
:10ADC00001202C4908700DE0402020490860002037
:10ADD0002849087006E040201C49091D0860102021
:10ADE000091F086024480078401E23490870FCF7BA
:10ADF000EBFC1420FAF7BFFE1F4800780028D5DCD2
:10AE00001B48B0F900301DA21E2101A802F04AFE25
:10AE1000012201A9002001F0ADFAFCF7D5FC462083
:10AE2000DFF864C000DF12480088401E00B21049FD
:10AE300008800F48B0F900000028B0DA202003494C
:10AE4000091D086000BFFEE731000020100C014022
:10AE500054727920746F205077724F66660000003C
:10AE60004154245143505752444E0D0A00000000F3
:10AE70004E00002051000020500000205077724FFB
:10AE80006666282564290000E5EE0008F0B5A7B045
:10AE900006460C464627BC4200DD3C4622460DA134
:10AEA00001A802F013FE00250AE0725D0CA16846BD
:10AEB00002F00CFE694601A8F9F724FA681CC5B235
:10AEC000A542F2DB012201A9002001F053FA27B0CC
:10AED000F0BD0000546370535B25645D3A000000D0
:10AEE000253032780000000029B1064A5269024339
:10AEF000044B5A6104E0034A52698243014B5A6190
:10AF0000704700000010024029B1064AD26902438E
:10AF1000044BDA6104E0034AD2698243014BDA61EF
:10AF2000704700000010024029B1064A126902432E
:10AF3000044B1A6104E0034A12698243014B1A610F
:10AF4000704700000010024029B1064A926902438E
:10AF5000044B9A6104E0034A92698243014B9A616F
:10AF6000704700000010024029B1064AD26802432F
:10AF7000044BDA6004E0034AD2688243014BDA6092
:10AF800070470000001002400348406A40F08070A3
:10AF900001494862704700000010024030B50021AE
:10AFA0000022002400232D4D6D6805F00C0121B115
:10AFB000042905D0082923D105E0294D056022E0A8
:10AFC000284D05601FE0254D6D6805F47012234D76
:10AFD0006D6805F48034022505EB92421CB9224DC0
:10AFE000554305600BE01D4D6D6815F4003F03D01F
:10AFF0001E4D5543056002E01A4D5543056002E0C1
:10B00000174D056000BF00BF144D6D6805F0F001DD
:10B010000909174D6B5C0568DD4045600F4D6D6893
:10B0200005F4E061090A124D6B5C4568DD408560FE
:10B030000A4D6D6805F46051C90A0D4D6B5C456899
:10B04000DD40C560054D6D6805F44041890B094D33
:10B050006B5CC568B5FBF3F5056130BD00100240BF
:10B0600000127A00001BB70000093D00808D5B00D4
:10B07000400100205001002010B5014600220023AD
:10B0800000204A11012A02D1094C236806E0022A55
:10B0900002D1074C236A01E0054C636A01F01F02EC
:10B0A000012494401C4201D0012000E0002010BD8A
:10B0B00000100240F0B50546002400230FE0E85AD6
:10B0C0002646671CBCB28855944206DA4FEA102C1B
:10B0D0002646671CBCB201F806C09E1CB3B2934260
:10B0E000EDDBF0BD10B5FBF774FD044694227E49FC
:10B0F0007E48FFF7DFFFA7227D497E48FFF7DAFF92
:10B10000794890F83100902803D17748007FA04219
:10B1100069D0012278A1002001F02CF99421724815
:10B12000F9F7E5F89020704981F83100052081F8A1
:10B130003200012081F83300FBF74BFD6A490877A4
:10B1400072A169482130F9F71BF940F2165066499F
:10B15000A1F82F007048C1F81D0070A1624874303A
:10B16000F9F70EF96FA160484430F9F709F971A1B8
:10B170005D485430F9F704F96EA15B486430F9F783
:10B18000FFF894225849594802F02EFCA72158484C
:10B19000F9F7ADF842F6D4105549A1F894000846E5
:10B1A00066490968016040F2D370514988800846B9
:10B1B00063490968C0F8061040F2D5704C494881CF
:10B1C000084660490968416140F273504849C881A6
:10B1D00008465D490968016140F26E504449888122
:10B1E00000F080FC59E04048B0F82F00A0F5A061C5
:10B1F000163952D045A13C482130F9F7C1F840F248
:10B2000016503949A1F82F00002081F8930000F072
:10B210007DFC37480078FF280BD135484078FF285F
:10B2200007D133488078FF2803D13148C078FF2800
:10B2300005D02F488088A0F57F41FF3907D12C48E1
:10B240003E490968016040F2D37029498880284846
:10B250008079FF280BD12648C079FF2807D12448E0
:10B26000007AFF2803D12248407AFF2805D02048E1
:10B270004089A0F57F41FF3908D11D483049096850
:10B28000C0F8061040F2D5701949488142F6D41032
:10B290001749A1F8940000F025FC01202B49087003
:10B2A000A72213491348FFF705FF11489630FBF713
:10B2B000F9FC0020254908700D48B0F89400A0F56D
:10B2C0002451D4390ED00CE00948B0F8941020A0D5
:10B2D00002F0D8FBFCF778FA4FF49670DFF88CC0D8
:10B2E00000DFF1E710BD00004C180020003C000812
:10B2F000E018002000FC0108526573657420436F5C
:10B300006E66696720506172616D21004853313269
:10B31000314C47310000000080D1F00863746E6545
:10B320007400000030303030303030303030303069
:10B3300030300000636172640000000088F800088B
:10B340008CF8000884F8000880F800081E0000202F
:10B35000466C61736853697A65436865636B206600
:10B3600061696C65643A25780D0A0000E5EE000815
:10B3700010B5012207A1002000F0FCFF094890F859
:10B38000930008B100F048FB0749D1F81D0001F017
:10B39000A1FA10BD526567697374726174696F6E4A
:10B3A00000000000E01800204C18002000B597B005
:10B3B00001203349087000203249087001203249C9
:10B3C00008603248D0F81D003149884204D32F4824
:10B3D000D0F81D00401C0BD101222EA1002000F04E
:10B3E000C9FF00222EA10120FDF786FA17B000BD8B
:10B3F0002648D0F81D10314A14A8FBF73DF9B8B122
:10B4000014AA2FA1684602F061FB0022694610468B
:10B4100000F0B0FF694614A8FEF740FB2CA0FDF732
:10B420000BFF6846FDF708FF30A0FDF705FF07E0BA
:10B4300001222FA1002000F09DFF31A0FDF7FCFEAE
:10B440001248D0F81D2039A114A802F03FFB14AA1D
:10B4500037A1684602F03AFB00226946104600F028
:10B4600089FF694614A8FEF719FB34A0FDF7E4FE36
:10B470006846FDF7E1FE36A0FDF7DEFE00BFB5E74A
:10B480006A0000202A000020140C01404C18002003
:10B490002058F20850534E204572726F72210000FE
:10B4A00044364435423643424231453042414335C9
:10B4B00042344544434546330000000076190020DD
:10B4C000436865636B436F64653D25730D0A000037
:10B4D00041542B4C53485454533D312C2244304159
:10B4E00033443145394332454200000032430000C5
:10B4F000436865636B436F64653D4E554C4C00007B
:10B5000041542B4C53485454533D312C2244304128
:10B510003344314539433245424242463143384152
:10B52000314341413742304443324300256C75007A
:10B5300050534E3D25730D0A00000000443644353B
:10B54000423643424231453043324542000000001A
:10B55000220D0A0010B5AEB001204D490870002040
:10B560004C49087001204C4908604CA0FDF764FE6E
:10B570004E48D0F81D204EA103A802F0A7FA03AA56
:10B580004CA106A802F0A2FA002206A9104600F07B
:10B59000F1FE06A903A8FEF781FA49A0FDF74CFECB
:10B5A00006A8FDF749FE782106A8F8F7A0FE49A0F5
:10B5B000FDF742FE4D48C07C4C49897C4B4A527C89
:10B5C000CDE9002102904948037C49A2282124A802
:10B5D00002F068FA002408E006AA02EB840124AA1B
:10B5E000105DFAF7BFF9601CC4B224A8F8F7B4FEE6
:10B5F000A042F1D806A8FDF71FFE40A0FDF71CFEF3
:10B600003A48C07D3949897D384A527DCDE90021CB
:10B6100002903648037D36A2282124A802F042FA7F
:10B62000002408E006AA02EB840124AA105DFAF7C0
:10B6300099F9601CC4B224A8F8F78EFEA042F1D894
:10B6400006A8FDF7F9FD782106A8F8F750FE32A00C
:10B65000FDF7F2FD2548C28933A124A802F036FA8D
:10B66000002408E006AA02EB840124AA105DFAF780
:10B6700079F9601CC4B224A8F8F76EFEA042F1D894
:10B6800006A8FDF7D9FD29A0FDF7D6FD2EB010BD07
:10B690006A0000202A000020140C014041542B4C69
:10B6A00053485454533D312C000000004C180020E6
:10B6B000256C750050534E3D25730D0A00000000A7
:10B6C00022443644354236434242314530433245C6
:10B6D000423243004244424242424242423746459D
:10B6E000434546314336463732430000E0180020D8
:10B6F00025642E25642E25642E25640032434236AF
:10B700004138434542424237464543454631433638
:10B71000463732430000000042364342424644412D
:10B72000424143353243000025640000220D0A00E7
:10B7300000B597B0064BA3F1510206A1684602F08E
:10B74000C5F9002269460120FDF7D6F817B000BD03
:10B750004F28002025733243324325730000000038
:10B7600010B58AB001202E49087000202D490870BC
:10B7700001202D4908602DA0FDF75EFD2FA0FDF7EB
:10B780005BFD02A933480068FBF756FB02A8FDF7F2
:10B7900053FD02A930480068FBF776FB02A8FDF7CD
:10B7A0004BFD2E488078C0F3C00020B12CA0FDF7DF
:10B7B00043FD202403E02EA0FDF73EFD1024304879
:10B7C000C0780A2817D02548007810F0010F04D15E
:10B7D0002CA0FDF731FD00240DE02048807810F00A
:10B7E000010F05D02CA0FDF727FD44F0010402E075
:10B7F0002FA0FDF721FD34A0FDF71EFD16480068BF
:10B80000CDE90004134831A21E21036802A802F00A
:10B8100049F9012202A9002000F0ACFD0AB010BDD8
:10B820006A0000202A000020140C014041542B4CD7
:10B8300053485454533D332C000000002233353715
:10B840003543463931374537363036353234423470
:10B85000450000002C000020C0000020B01D00208A
:10B86000463235443734393234333637000000003D
:10B87000324136373734393234333637000000003E
:10B88000EB0000204530363534373030353030303D
:10B890003533303000000000313735333936363239
:10B8A00046323544394135423444344600000000C4
:10B8B0003137353339363632324136373941354210
:10B8C0003444344600000000220D0A0056626174C0
:10B8D0003D25642C4353513D25642C4750533D2551
:10B8E0003032780000B5A9B001202249087000204C
:10B8F0002149087021A110A802F0E8F82448B0F806
:10B900002F2024A101A802F0E1F806A901A8F9F767
:10B910007FFC06A910A8F8F7F5FC1FA110A8F8F7FE
:10B92000F1FC23480368234823A1026801A802F020
:10B93000CDF806A901A8F9F76BFC06A910A8F8F73D
:10B94000E1FC002210A90120FCF7D6FF184800688E
:10B9500000900F48B0F82F20164819A1036810A8CE
:10B9600002F0B4F8012210A9002000F003FD29B074
:10B9700000BD00006A0000202A0000204433413648
:10B98000443343334230453642314245324300006E
:10B990004C180020256400003243433441334246B2
:10B9A00045394230453642314245324300000000BD
:10B9B000B8000020B400002025642C25640000009D
:10B9C000415665723D25642C4D5665723D25642CAB
:10B9D000505665723D25640010B5012204A1002077
:10B9E00000F0C8FC0120064981F8300110BD0000BC
:10B9F0005265736574204D6F64656D210000000011
:10BA0000D8270020024A1080024A116070470000C7
:10BA1000460000204800002010B500240FE009492E
:10BA200001EB84020849022303FB041007A1F8F785
:10BA3000C5FC044810F8240005490855641C062C70
:10BA4000EDDB10BD1038002067190020253278008A
:10BA50002D0100202DE9F04118480078012803D07D
:10BA600016480078022826D11448B0F8961114A080
:10BA700002F008F8114D6D1D00240FE0A01C2E5C93
:10BA8000E01C2F5C295DA01C2954601C295CE01C73
:10BA900029542E55601C2F54201D84B20748B0F83D
:10BAA0009601A042EADC012229460320FCF724FF8C
:10BAB000002002490870BDE8F08100002435002014
:10BAC0005454535F4C454E3A25640D0A0000000063
:10BAD00010B54FF4CC710248F8F709FC10BD000016
:10BAE0002435002010B5202005490860A72205490B
:10BAF000054801F079FF20200149091D086010BDAB
:10BB0000100C0140E018002000FC010810B52020B6
:10BB10000549086094220549054801F065FF202089
:10BB20000149091D086010BD100C01404C1800208F
:10BB3000003C000870B50446002525465E480078A4
:10BB400085422FD05C4805700078062828D2DFE8AF
:10BB500000F003090F151B21012258A10320FCF757
:10BB6000CBFE1EE001225AA10320FCF7C5FE18E01F
:10BB700001225CA10320FCF7BFFE12E001225EA1BE
:10BB80000320FCF7B9FE0CE0012260A10320FCF7C2
:10BB9000B3FE06E0012265A10320FCF7ADFE00E044
:10BBA00000BF00BF68480078012877D1424800787C
:10BBB000664981F89300FFF7A9FF3F4800780628FF
:10BBC00076D2DFE800F0031527394C5F60A0FDF75F
:10BBD00033FB0120DFF890C100DFFAF755FF0122A7
:10BBE00062A10320FCF788FE00205749087060E03E
:10BBF00057A0FDF721FB0120DFF86CC100DFFAF749
:10BC000043FF012260A10320FCF776FE00204E498D
:10BC100008704EE04EA0FDF70FFB0120DFF848C191
:10BC200000DFFAF731FF01225EA10320FCF764FE7A
:10BC30000020454908703CE061A0FDF7FDFA0120B5
:10BC4000DFF824C100DF64A0FDF7F6FA012266A147
:10BC50000320FCF751FE00203B49087029E069A051
:10BC6000FDF7EAFA0120DFF800C100DF5AA0FDF776
:10BC7000E3FA012269A10320FCF73EFE00203249CD
:10BC8000087016E06FA0FDF7D7FA0120DFF8D8C0E2
:10BC900000DF51A0FDF7D0FA012201E00AE007E041
:10BCA0006EA10320FCF728FE00202749087000E061
:10BCB00000BF00BF70BD000067000020353137466F
:10BCC00044433745454138314138353200000000A2
:10BCD00038433445323139453231364130463546C4
:10BCE00000000000303934453231394532313641B7
:10BCF0003046354600000000444235363231394581
:10BD00004541383141383532000000004442353673
:10BD100032313945333130303338303033303030F0
:10BD2000333030303436353100000000444235368F
:10BD300032313945333830303330303033303030D1
:10BD40003436353100000000290000204C18002056
:10BD500041542B4C43544D4F4241505245463D3285
:10BD60002C300D0A00000000E5EE00084442384681
:10BD7000363535313531374644433745454138311D
:10BD800041383532000000004442384636353531FE
:10BD90003843344532313945323136413046354603
:10BDA00000000000444238463635353130393445DC
:10BDB00032313945323136413046354600000000D7
:10BDC00041542B4C43544D4F4241505245463D3512
:10BDD0002C300D0A0000000041542B4D4F444F44BD
:10BDE0005245583D350D0A00444238463635353106
:10BDF00044423536323139454541383141383532A2
:10BE00000000000041542B4C43544D4F42415052CE
:10BE100045463D352C360D0A0000000044423846A8
:10BE200036353531444235363231394533313030AB
:10BE300033383030333030303330303034363531E1
:10BE40000000000041542B4C43544D4F424150528E
:10BE500045463D352C380D0A000000004442384666
:10BE60003635353144423536323139453338303064
:10BE7000333030303330303034363531000000006C
:10BE800070B588B005460E461B4890FBF5F084B2AD
:10BE9000ADF818400320ADF814000020ADF81A00EA
:10BEA000ADF816008DF81C0005A9144800F064FBDD
:10BEB0007020ADF80400204604EBD0714910ADF8B5
:10BEC0000A100120ADF806000220ADF80C0001A90F
:10BED0000A4800F0F1FA0821084800F03FFB012170
:10BEE000064800F0DDFAB0B20121DFF814C000DF2F
:10BEF0000449086008B070BD808D5B0000080040F8
:10BF00007DF500082000002070B588B005460E467B
:10BF100079210720FFF776FD1F4890FBF5F084B2EA
:10BF2000ADF818400320ADF814000020ADF81A0059
:10BF3000ADF816008DF81C0005A9184800F01CFB90
:10BF400083210720FFF75EFD7020ADF80400204636
:10BF500004EBD0714910ADF80A100120ADF80600CD
:10BF60000220ADF80C0001A90C4800F0A5FA082148
:10BF70000A4800F0F3FA8E210720FFF743FD012164
:10BF8000064800F08DFAB0B2F9F7F5FD002103483C
:10BF900000F086FA08B070BD808D5B00000800409C
:10BFA00043185A00FF2A00DD7047034B1870034BFB
:10BFB000197000BFF8E7000076000020770000202D
:10BFC0002DE9F041224844788578C6780779302CED
:10BFD00013D1302D11D1322E0FD1302F0DD1B0F819
:10BFE0009601001F1A49A1F896010120087001224C
:10BFF00018A1002000F0BEF928E0012C10D1022D7C
:10C000000ED11348B0F89601001F1149A1F896010E
:10C0100002200870012211A1002000F0ABF915E008
:10C02000202C13D1202D11D1202E0FD1202F0DD156
:10C0300001220DA1002000F09DF90548B0F89601FD
:10C04000001F0349A1F8960100200870BDE8F081A7
:10C0500024350020537461727400000050757265BD
:10C0600020545453000000006E6F742068616E64A9
:10C070006C65000010B50446062C2ED2DFE804F0F3
:10C08000030A11181F26002015490870012000F02E
:10C0900029F822E0012012490870052000F022F85A
:10C0A0001BE002200E490870062000F01BF814E087
:10C0B00003200B490870042000F014F80DE0042060
:10C0C00007490870012000F00DF806E0042004493B
:10C0D0000870022000F006F800BF00BF10BD00008D
:10C0E0008900002010B504460A2C60D2DFE804F075
:10C0F000050E172029323B444D560021084600F01A
:10C1000059F800210846FFF74BFF50E000210120BD
:10C1100000F050F800210846FFF742FF47E00121F8
:10C12000084600F047F800210846FFF739FF3EE0D7
:10C130000A21012000F03EF800210846FFF730FFF9
:10C1400035E00021084600F035F800210120FFF716
:10C1500027FF2CE00021084600F02CF801210846BA
:10C16000FFF71EFF23E00021084600F023F80A2114
:10C170000120FFF715FF1AE00021012000F01AF856
:10C1800000210120FFF70CFF11E00121084600F01B
:10C1900011F801210846FFF703FF08E00A210120FA
:10C1A00000F008F80A210120FFF7FAFE00BF00BFE7
:10C1B00010BD000043185A00FF2A00DD7047034BF2
:10C1C0001870034B197000BFF8E7000074000020DE
:10C1D0007500002010B500F001F810BD0CB500206E
:10C1E000019000903248006840F480303049086087
:10C1F00000BF2F48006800F4003000900198401CF8
:10C200000190009818B90198B0F5A06FF1D12848B5
:10C21000006810F4003F02D00120009001E00020EF
:10C220000090009801283FD12248006840F010009B
:10C23000204908600846006820F0030008600846AE
:10C24000006808601A484068194948600846406814
:10C2500048600846406848600846406820F47C1002
:10C2600048600846406840F430204860084600684E
:10C2700040F08070086000BF0D48006810F0007F3B
:10C28000FAD00B48406820F003000949486008468E
:10C29000406840F00200486000BF0548406800F078
:10C2A0000C000828F9D101E000BFFEE70CBD00003A
:10C2B0000010024000200240012223A1002000F0D3
:10C2C00059F8102023490860402008600120091F08
:10C2D0000860022020490860C0021E49091F08604A
:10C2E0004000091D08604000091F086040F6B83092
:10C2F000FBF746FA002144F21C00FEF725FE002160
:10C300004FF4C020FEF700FE00211448F8F7D8FED5
:10C3100000210120FEF7E8FD11480068DFF844C065
:10C3200000DF11480068DFF83CC000DF0F480068FC
:10C33000DFF830C000DF06E04FF47A70DFF830C07D
:10C3400000DFFBF741FAF7E7536C656570696E67CC
:10C3500000000000140C01401008014000240140BE
:10C36000F4000020A1F60008F000002034010020B5
:10C37000E5EE00082DE9F04104460D461646012C75
:10C3800001D1BDE8F0810948007800B1F9E72846FD
:10C39000F7F7E2FF07463946284600F08DFE1EB14A
:10C3A000022103A000F088FE00BFEAE7040000209D
:10C3B0000D0A000018B10121034A116003E00121B8
:10C3C000014A121F11607047140C014008B501208A
:10C3D000ADF8000010208DF8030003208DF8020056
:10C3E00069460348FAF73EF80020FFF7E3FF08BD6F
:10C3F000000C014010B51248006840F001001049DF
:10C400000860084640680F4908400D4948600846E2
:10C4100000680D4908400A4908600846006820F491
:10C42000802008600846406820F4FE0048604FF411
:10C430001F008860FFF7CEFE04480549086010BD64
:10C44000001002400000FFF8FFFFF6FE0040000869
:10C4500008ED00E001220AA10020FFF78BFF0C4845
:10C460000068DFF830C000DF0B480068DFF824C048
:10C4700000DF0A480068DFF81CC000DF00BFFEE7ED
:10C4800053797354656D2052657365742100000003
:10C49000F4000020A1F60008F00000203401002084
:10C4A00021B1028842F00102028004E002884FF6C6
:10C4B000FE731A400280704770B5002400220023EA
:10C4C000058C4FF6EF7635400584028C8388048B0B
:10C4D00048F6FF752C404FF6FF452C400D884FF66F
:10C4E000FF7606EA05252C434FF6DF752A400D89B5
:10C4F00006EA05152A434D8806EA05152A43154D17
:10C50000A84202D0144DA8421DD14FF67F752A4093
:10C510004D894FF6FF7606EA05152A434FF6BF759B
:10C520002A408D8806EA05152A434FF6FF352B4031
:10C530004FF2FF752B408D8906EA85052B43CD8987
:10C5400006EA85052B4383800483CD880587028412
:10C5500070BD0000002C0140003401400A4600215B
:10C56000018B4FF2FF7319404FF6FF7303EA02236A
:10C570001943018370470000002202881D4B984236
:10C580000ED01D4B98420BD0B0F1804F08D01B4B02
:10C59000984205D01A4B984202D01A4B984204D1C7
:10C5A0004FF68F731A404B881A43174B984207D0A7
:10C5B000164B984204D04FF6FF431A40CB881A43DB
:10C5C00002808B8883850B8803850A4B98420BD0A9
:10C5D000094B984208D00E4B984205D00D4B98421B
:10C5E00002D00D4B984201D10B7A0386012383823E
:10C5F00070470000002C014000340140000400405E
:10C6000000080040000C00400010004000140040F2
:10C6100000400140004401400048014010B502467E
:10C620000B465078012103E04C1C145D6040491C0E
:10C630005C1E8C42F8DC10BD10B5084C1C21204655
:10C64000F7F755FE064C68212046F7F750FE2046C6
:10C65000807820F008002146887010BD283800201E
:10C66000B01D00202DE9F04F89B007468B4691465A
:10C670009A46DDF848803D460020079000240120BE
:10C6800006900020059008F1060080B2019008F1A4
:10C690000C0080B200905A463BA102A801F016FAA5
:10C6A0007E222046641C2A544FEA19222046641C2C
:10C6B0002A542046641C05F8009000203449087173
:10C6C0000846C0F8088002792046641C2A540846AF
:10C6D000027A2046641C2A542E4890F893000128C0
:10C6E00014D000222046641C2A5400260BE002A825
:10C6F000815D02AA701C105C61F31F10C2B220465B
:10C70000641C2A54B61C0A2EF1DB09E0002605E061
:10C710002148825D2046641C2A54761C062EF7DBD5
:10C720001E480088020A2046641C2A541B480278CE
:10C730002046641C2A5419480088401C1749088068
:10C74000BAF1000F09D0002605E01AF806202046AD
:10C75000641C2A54761C4645F7DB21462846FFF721
:10C760005DFF08902146641C08986854611E681C8F
:10C7700001F08AFE0446641C7E222046641C2A5472
:10C78000204609B0BDE8F08F25303130750000003B
:10C7900074380020E01800202D0100201E01002028
:10C7A00010B59AB000F018F81C2000900848D0F896
:10C7B0001D10084B4FF4007201A8FFF753FF84B21D
:10C7C000224601A90120FBF745FD1AB010BD00006B
:10C7D0004C1800202838002010B53C48C0793C494E
:10C7E00088753A48017A3A48C1753848417A3848DC
:10C7F00001763648817A364841763448C17A3448E1
:10C8000081763248017B3248C17600203049086089
:10C810002E48807810F0010F0FD00846406840F095
:10C82000807048600846406840F0007048600846E4
:10C83000406840F08050486002E000202449486091
:10C840002248008FC0F30720204991F8381040EAB1
:10C8500001201F4908821D48008BC0F307201B4997
:10C86000097E40EA01201A4948821848808B888254
:10C870000120F9F779FF1548406E000E144908723F
:10C880001248406E010C124841721048B0F8640022
:10C89000010A0F4881720D4890F864100C48C1726B
:10C8A0000A48006E000E0A4908730848006E010C21
:10C8B000074841730548B0F86000010A04488173D5
:10C8C000024890F860100248C17310BDB01D0020EE
:10C8D0002838002070B59AB0054600202449088009
:10C8E0004880002404E000212148001D0155641CFB
:10C8F000052CF8DB002404E000211D480930015517
:10C90000641C142CF8DB280E19494877290C1848A8
:10C910008177290AC17780F82050002405E00022A1
:10C9200013481D30211D4254641C032CF7DB0020EA
:10C930000F4981F82400002404E000210C48253030
:10C940000155641C082CF8DB2E2000900948D0F813
:10C950001D10074B4FF4807201A8FFF783FE86B2CB
:10C96000324601A90120FBF775FC1AB070BD00002A
:10C97000443800204C18002010B59AB000200090D8
:10C980000748D0F81D100023022201A8FFF76AFE15
:10C9900084B2224601A90120FBF75CFC1AB010BD4D
:10C9A0004C1800206A210948F7F7A1FC002108482B
:10C9B000DFF820C000DF07E04FF6FF710448DFF822
:10C9C00018C000DFFBF7D4FBF6E700002839002091
:10C9D00038010020D5F200084DF3000838B50024D6
:10C9E00040F225512D4800F0E4F9002848D02B48AA
:10C9F00000F09AFAC0B2009040F22551274800F0AA
:10CA000062F927480078022805D19DF800102548D2
:10CA100000F08FFA34E022480078012805D19DF813
:10CA20000010214800F085FA2AE02048008838BB31
:10CA30009DF800101E4802880088401C1C4B18807E
:10CA40001C48815418460088C82802DB002019467B
:10CA500008801748008802280EDB174800780D2848
:10CA60000AD19DF800000A2806D1114800880F4914
:10CA7000088000200E4908809DF800000E490870CB
:10CA80000821064800F088F9012806D1034800F083
:10CA90004BFA0821014800F00DF938BD003801407B
:10CAA0000400002000440040004800400C0000202A
:10CAB0000A000020CC0900200700002008B540F241
:10CAC00025512E4800F075F9002848D02B4800F079
:10CAD0002BFAC0B200902A48007802280AD19DF8AB
:10CAE0000010284800F025FA40F22551234800F0B4
:10CAF000EAF808BD2248007801280AD19DF8001004
:10CB0000204800F016FA40F225511C4800F0DBF8EE
:10CB1000EFE71D48008840F21441884217DA9DF87B
:10CB200000001A491A4A1288885419480088401C83
:10CB300080B21749088040F21441884202DB00208D
:10CB40001349088010480088401C0F49088011488C
:10CB500001F012FD40F22551084800F0B4F8082118
:10CB6000064800F019F9012806D1044800F0DCF964
:10CB70000821024800F09EF800BFBAE700440040D8
:10CB8000040000200038014012000020940A002018
:10CB9000140000200401002038B5002440F2255183
:10CBA000374800F006F900285BD0354800F0BCF9A2
:10CBB000C0B2009033480078012805D19DF80010DC
:10CBC000314800F0B6F943E03048008800283CD1F5
:10CBD0009DF800002E492F4A128888540846007894
:10CBE000242803D000202B49088004E0294800882D
:10CBF000401C2849088027480088C72802DB0020FD
:10CC000024490880244800780D2821D19DF800008F
:10CC10000A281DD11E484078472812D11C48C078E8
:10CC200052280ED11A48407943280AD100211948C8
:10CC30000088401E164A115416480088134908807F
:10CC400006E000201349088002E000201149088016
:10CC500040F225510A4800F036F89DF800000E49D0
:10CC600008700821064800F097F8012806D104480A
:10CC700000F05AF90821024800F01CF838BD000005
:10CC80000048004004000020003801401A00002045
:10CC9000A80E00201C0000200600002010B5FFF7A1
:10CCA0009DFE10BD10B5FFF709FF10BD10B5FFF7D1
:10CCB00073FF10BD01F40072B2F5007F00D100BF18
:10CCC000CA430280704710B500220023A1F510640A
:10CCD0006A3C00D100BF0A1201249440A3B2DC4395
:10CCE000048010BD21B1828942F40052828104E0A7
:10CCF00082894DF6FF731A408281704710B5044651
:10CD00002048844209D101218803FEF72DF9002132
:10CD10004FF48040FEF728F932E01B48844209D1E5
:10CD200001214804FEF700F900214FF40030FEF71E
:10CD3000FBF825E01548844209D101218804FEF75B
:10CD4000F3F800214FF48020FEF7EEF818E01048C9
:10CD5000844209D10121C804FEF7E6F800214FF40E
:10CD60000020FEF7E1F80BE00A48844208D10121D7
:10CD70000805FEF7D9F800214FF48010FEF7D4F82B
:10CD800010BD000000380140004400400048004051
:10CD9000004C00400050004002460020B1F5007FEA
:10CDA00000D100BF13880B4201D0012000E0002019
:10CDB000704770B502460024002300250020A1F52D
:10CDC00010666A3E00D100BFC1F3421501F01F0397
:10CDD000012606FA03F3012D02D19689334006E0BD
:10CDE000022D02D1168A334001E0968A33400C129C
:10CDF000012606FA04F41688344013B10CB1012060
:10CE000000E0002070BDF0B5034600240026002598
:10CE10000020A1F510676A3F00D100BF1846C1F39A
:10CE2000421401F01F06012707FA06F5012C01D173
:10CE30000C3004E0022C01D1103000E014301AB1A3
:10CE400007682F43076002E00768AF430760F0BD43
:10CE50002DE9F04786B005460E460024A24600BFE5
:10CE6000A1460027B08900B100BF2F462C8A4CF69E
:10CE7000FF700440F08804432C82AC894EF6F31016
:10CE80000440B08831890843718908430443AC8168
:10CE9000AC8A4FF6FF400440B0890443AC8201A83D
:10CEA000FEF77CF81F48874202D1DDF810A001E0B0
:10CEB000DDF80CA0A88910F4004F08D00AEBCA00D6
:10CEC00000EB0A1031684900B0FBF1F807E00AEB0B
:10CED000CA0000EB0A1031688900B0FBF1F8642049
:10CEE000B8FBF0F004012009642101FB1089A88936
:10CEF00010F4004F08D0322000EBC900B0FBF1F075
:10CF000000F00700044308E0322000EB0910642120
:10CF1000B0FBF1F000F00F0004432C8106B0BDE837
:10CF2000F08700000038014001468888C0F30800FF
:10CF30007047C1F3080282807047000000B585B0D9
:10CF4000012144F20400FDF7FFFF4FF40070ADF83B
:10CF5000100018208DF8130003208DF8120004A98A
:10CF60002448F9F77FFA4FF48060ADF810000420F0
:10CF70008DF8130003208DF8120004A91D48F9F75D
:10CF800071FA4FF4E13000900020ADF80400ADF8E4
:10CF90000600ADF80800ADF80C000820ADF80A0056
:10CFA00069461548FFF754FF01211348FFF79AFE21
:10CFB00040211148FFF77EFE002240F227710E4803
:10CFC000FFF721FF002240F225510B48FFF71BFF1E
:10CFD000002240F224410848FFF715FF00200749CE
:10CFE000088007490880074908700749087005B09C
:10CFF00000BD000000080140003801400A00002088
:10D000000C0000200E000020050000201FB5044683
:10D0100027480078A04202D025490C7000E01FBDCF
:10D020002448FFF76BFE1CB34FF4E1300090002062
:10D03000ADF80400ADF80600ADF80800ADF80C003E
:10D040000C20ADF80A0069461A48FFF701FF0121DC
:10D050001848FFF747FE012240F225511548FFF717
:10D06000D2FE002240F224411248FFF7CCFE1CE021
:10D070004FF4E13000900020ADF80400ADF8060058
:10D08000ADF80800ADF80C000820ADF80A006946BC
:10D090000848FFF7DDFE01210648FFF723FE0022C6
:10D0A00040F225510348FFF7AEFE00BFB7E700008E
:10D0B000080000200038014070B505460E460024E7
:10D0C0000BE0295D0648FFF734FF00BF402104480C
:10D0D000FFF762FE0028F9D0641CB442F1DB70BD9A
:10D0E0000038014000B585B001210420FDF72CFF78
:10D0F00001214804FDF708FF0820ADF81000482082
:10D100008DF8130003208DF8120004A92A48F9F7BE
:10D11000A9F90420ADF8100018208DF8130004A917
:10D120002548F9F79FF94FF4E13000900020ADF861
:10D130000400ADF80600ADF80800ADF80C000C20B6
:10D14000ADF80A0069461D48FFF782FE40211B48E2
:10D15000FFF7B0FD002240F227711848FFF753FE99
:10D16000012240F225511548FFF74DFE002240F202
:10D1700024411248FFF747FE012228210F48FFF7FC
:10D1800042FE012260210D48FFF73DFE01210B48C0
:10D19000FFF7A8FD00200A4908800A4908800A49CB
:10D1A00008800A4908800A49087040F21441094879
:10D1B000F7F79DF805B000BD0008014000440040AD
:10D1C0001000002012000020140000201600002093
:10D1D00018000020940A00202DE9F04788B0DA48B2
:10D1E0000088082802DA08B0BDE8F087D648008831
:10D1F00040F21241884218DD002240F22551D34806
:10D20000FFF701FE0020D2490880CF490880D149AC
:10D210000880012240F22551CC48FFF7F4FD01229D
:10D22000CDA11046FFF7A6F8DDE7C7480688042E13
:10D2300000DAD8E7102E01DA354600E01025C5489F
:10D24000078800240DE0C848C05D03A90855781C74
:10D2500080B2074640F21441884200DD0027601C7E
:10D2600084B2AC42EFDBAD210420FEF7CBFBBFA1C3
:10D2700003A8FCF773F800287ED0B648078800247E
:10D280000EE0B948C05D0A2800D10BE0781C80B2DE
:10D29000074640F21441884200DB0027601C84B23C
:10D2A000B442EEDB00BFB44267DA601C85B2BE2137
:10D2B0000420FEF7A7FB40F21240854245DAAE4853
:10D2C0000580002415E0A848A2490988415CAA48C5
:10D2D000801C01559F480088401C80B29D490880F1
:10D2E00040F21441884202DB00209A490880601C09
:10D2F00084B2AC42E7DB00219F48801C015500222C
:10D3000040F225519148FFF77EFD8F480088401B71
:10D310008D490880012240F225518C48FFF773FDAA
:10D32000CC210420FEF76EFB93480088401C9249F4
:10D33000088008460188801CFCF716FB20B10122FA
:10D340008EA10020FFF716F84DE78B4805800024DA
:10D350001EE085487F49098810F8019040F212408C
:10D36000844203DA8448801C00F8049079480088DD
:10D37000401C80B2774901E032E030E0088040F2A2
:10D380001441884202DB002072490880601C84B28C
:10D39000AC42DEDB0021784880F81514002240F210
:10D3A00025516A48FFF72FFD67480088401B6649F2
:10D3B0000880012240F225516448FFF724FDDF2157
:10D3C0000420FEF71FFB6C480188801CFCF7CCFA98
:10D3D00020B101226DA10020FEF7CCFF03E702E798
:10D3E000102E00DAFFE65B4807884FF0000AD046AF
:10D3F000002425E05C4810F80790B9F12C0F08D103
:10D40000BAF1010F04DA0AF1010000F0FF0A0DE0A1
:10D4100018E0BAF1010F09D1B8F1040F06DA40465D
:10D42000411C1FFA81F801A901F80090781C80B214
:10D43000074640F21441884200DB0027601C84B29A
:10D44000B442D7DB00BFB44200DBCCE6FA210420B3
:10D45000FEF7D8FA002001A901F8080001A8F7F7A3
:10D46000A9F885B20A2D02DA4FF001080CE0642D0C
:10D4700002DA4FF0020807E0B5F57A7F02DA4FF0E2
:10D48000030801E04FF0040805EB08000E3085B2F8
:10D49000AE4200DAA7E640F21240854241DA364851
:10D4A0000580002415E030482A490988415C32484B
:10D4B000801C015527480088401C80B225490880FF
:10D4C00040F21441884202DB002022490880601C9F
:10D4D00084B2AC42E7DB00212748801C01550022C2
:10D4E00040F225511948FFF78EFC17480088401B71
:10D4F00015490880012240F225511448FFF783FCAA
:10D500001D480088401C1C49088008460188801C72
:10D51000FCF72AFA80B1012220A10020FEF72AFFA1
:10D520000AE0224621A103A800F0D0FA012203A9B3
:10D530000020FEF71FFF56E640F21B110420FEF705
:10D5400061FA00BF4FE600001200002000440040D6
:10D5500014000020160000205B52783242756620CD
:10D560004F7665725D000000940A00202B544350F2
:10D570005245435600000000A00100204D51756542
:10D5800075652046756C6C31000000004D51756565
:10D5900075652046756C6C32000000004D51756554
:10D5A00075652046756C6C330000000041744D7346
:10D5B00067427566204F766572205B25755D0000B9
:10D5C00070B505460E4600240BE0295D0648FFF7BE
:10D5D000B0FC00BF40210448FFF7DEFB0028F9D073
:10D5E000641CB442F1DB70BD0044004000B585B05E
:10D5F00001210820FDF7A8FC01218804FDF784FC27
:10D600004FF40060ADF8100048208DF8130003209F
:10D610008DF8120004A91948F8F724FF4FF41650AA
:10D6200000900020ADF80400ADF80600ADF8080049
:10D63000ADF80C000420ADF80A0069461048FFF769
:10D6400007FC40210E48FFF735FB012240F225512F
:10D650000B48FFF7D8FB002240F227710848FFF77C
:10D66000D2FB01210648FFF73DFBC8210548F6F72C
:10D670003EFE00200449088005B000BD000C0140BA
:10D6800000480040A80E00201A000020704700004B
:10D6900000B599B0002214A10120FBF72DF9FAF78B
:10D6A00093F86420DFF854C000DFFAF78DF86420A7
:10D6B000DFF848C000DF812042214D227823CDE9E8
:10D6C0000032CDE902100E480E4A5021036805A829
:10D6D00000F0E8F905A8FBF7AFFD01220AA1002040
:10D6E000FEF748FE19B000BD443546444434444179
:10D6F000433946444243423600000000E5EE00084C
:10D70000B800002080F900085570646174652050ED
:10D710004F432100632803D0002806DB1F2804DCC8
:10D720001B491C4A127841F822001B490978491C00
:10D73000194A117017490978012903D0114609784F
:10D74000022923D112490968002908DB1049096818
:10D750001F2904DC0E490968104A11600FE00C49CA
:10D760004968002908DB0A4949681F2904DC08497F
:10D7700049680A4A116002E06321084A1160632186
:10D78000034A116051600021034A11707047000084
:10D79000DC000020D1000020D8000020C0000020C4
:10D7A000044802680448018804A000F06BF900BF37
:10D7B000FEE7000048000020460000200D0A5B55EF
:10D7C00046485D463D25642C4C3D25640000000024
:10D7D00070B51B4C1BA0FBF72FFD002526E064262F
:10D7E00021A0FBF729FD1AE040F21441A01CFCF730
:10D7F0001BF8208078B124A1A01CFBF7AFFD28B94D
:10D80000012222A10020FEF7B5FD70BD3EB90DA09A
:10D81000FBF712FD03E00120DFF884C000DF3000D9
:10D82000A6F10101CEB2DFD1681CC5B20A2DD6DB4C
:10D8300001221CA10020FEF79DFD00BFE5E70000CE
:10D84000B605002061742B737973636D643D737446
:10D850006172745F70636D20766F6C756D652036D4
:10D8600020370D0A0000000061742B737973636D1B
:10D87000643D73746172745F70636D20766F6C7554
:10D880006D650D0A00000000362037005B30375D03
:10D8900053657420566F6C756D65206F6B000000CA
:10D8A000E5EE00085B30375D53657420566F6C758C
:10D8B0006D65206661696C656400000070B51B4C85
:10D8C00000221BA11046FEF755FD002525E032265B
:10D8D0001BA0FBF7B1FC1BE040F21441A01CFBF7BE
:10D8E000A3FF208080B118A1A01CFBF737FD20B159
:10D8F00016A1A01CFBF732FD50B9012216A1002091
:10D90000FEF738FD002070BD0120DFF854C000DFB5
:10D910003000A6F10106DFD16D1C642DD7DB01229A
:10D9200010A10020FEF726FD0120ECE7B60500203F
:10D93000576169744D6F64656D52756E3A000000F1
:10D94000415445300D0A00004F4B00002B504F430F
:10D950003A5354415254000052756E696E6700008C
:10D96000E5EE000854696D654F7574001B484078FA
:10D9700000B9704719480078012806D100201749DE
:10D9800081F82D0181F82E01F3E7DFF854C000DFA4
:10D9900014490968884200D2EBE7DFF844C000DF91
:10D9A0006430104908600D4890F82D01FA2806DA15
:10D9B0000A4890F82D01401C084981F82D010748BC
:10D9C00090F82E01FA2806DA044890F82E01401C3F
:10D9D000024981F82E0100BFCBE70000D8270020C4
:10D9E00071F50008000100202DE9F04705460E46BC
:10D9F000904633210620FEF705F8B5F1006F02D3FB
:10DA00001F48854201D3BDE8F087A805800D00D0EE
:10DA1000F9E737210620FDF7F5FFF8F72BFC392150
:10DA20000620FDF7EFFF2846F8F7BAFB0746042F5C
:10DA300004D03C210620FDF7E5FFE4E73F21062066
:10DA4000FDF7E0FF00240CE0315D601C305C01EB71
:10DA500000201FFA80F928194946F8F7EBFBA01CB3
:10DA600084B24445F0DB47210620FDF7CBFFF8F7F1
:10DA7000D7FB49210620FDF7C5FF00BFC3E7000023
:10DA8000000002080FB4054B10B503A9044A029820
:10DA900000F016F910BC5DF814FB000005E5000865
:10DAA000900100200FB41CB50A46521ECDE90002B9
:10DAB00007A9054B6A46069800F002F9009A002172
:10DAC00011701CBC5DF814FB07E400080FB4084B90
:10DAD00010B504A902AA039800F0F2F8044602A9BE
:10DAE000002000F09BFC204610BC5DF814FB0000F9
:10DAF0001DE40008004870479C01002002E008C8AF
:10DB0000121F08C1002AFAD170477047002001E0B7
:10DB100001C1121F002AFBD1704700002DE9FF5FF1
:10DB2000DDE90220010DDDF838B0024310D10F9875
:10DB300001244CA2012808D0002100980F9BC0E9C5
:10DB40000021C0E90243BDE8FF9F6FEA0B01F4E743
:10DB5000A1F2FF3144F6105041430D140F980128F3
:10DB60000ED0A5EB0B00401C4FF000043E4EDFF83A
:10DB7000FC90B0F1000AA04605DACAF1000717E0F0
:10DB8000CBF10000F0E7074612E0F80707D0224685
:10DB9000334640464946F6F7CEFD80468946224642
:10DBA000334610461946F6F7C6FD04460E467F106A
:10DBB000002FEAD1DDE90201BAF1000F42464B46DF
:10DBC00002DAF6F7B8FD01E0F6F727FE04460E4646
:10DBD0000022274BF7F74EF803D84FF0FF300146ED
:10DBE00007E00022234B20463146F6F7FDFCF7F70D
:10DBF00029F8102409E0002C0ADB0A220023F6F79A
:10DC0000BBFE019B30321A55641E50EA0102F2D16C
:10DC1000641C019AC4F1110314440F9A012A09D01B
:10DC20000122084301D15B450FDD4FF0000205F1F1
:10DC300001050DE0084303D1A3EB0B056D1E09E0C0
:10DC400000204FF0110B0F9088E701DA00226D1EC3
:10DC5000002A83D000980F99C0E90231C0E900453D
:10DC600071E7000030000000000024400000F03F99
:10DC70000000F0430000E03F10B5002A06DA22F071
:10DC80000042D21D22F00703102203E0D21C22F032
:10DC900003030C2213B19C188C4201D9012010BD42
:10DCA000024401448360C0E90021C91AD0188842A7
:10DCB00002D810600246F9E70020106010BD000095
:10DCC0002DE9FF4F95B09B4689460646002512E296
:10DCD000252878D10024761CF94A2746012105948D
:10DCE0003378203B01FA03F0104202D00443761C43
:10DCF000F6E730782A2811D06FF02F033078A0F1A2
:10DD00003002092A16D8059A44F0020402EB820276
:10DD100003EB42021044761C0590EFE759F8042B00
:10DD20000592002A03DA504244F40054059044F06E
:10DD30000204761C30782E2816D116F8010F44F014
:10DD400004042A280DD06FF02F023078A0F13003A0
:10DD5000092B09D807EB870302EB4303C718761C8E
:10DD6000F3E759F8047B761C30786C280FD006DC7A
:10DD70004C2817D068280DD06A2814D104E07428E4
:10DD800010D07A280FD10DE044F400140AE044F4D6
:10DD9000801401E044F440147278824202D1761C6F
:10DDA00004F58014761C307866280BD013DC5828D4
:10DDB00077D009DC002875D04528F6D04628F4D065
:10DDC00047281AD19FE118E0632835D0642879D01C
:10DDD000652812D197E1702873D008DC6728F1D04C
:10DDE00069286FD06E280DD06F2806D1B5E0732852
:10DDF0002CD0752875D0782874D05A46179990473A
:10DE00006D1C76E1C4F30250022809D003280DD01E
:10DE1000D9F8001004280DD00D6009F1040968E15B
:10DE2000D9F80010EA17C1E90052F6E7D9F8001056
:10DE30000D80F2E70D70F0E719F8041B8DF8001063
:10DE400000208DF80100EA46012003E059F804ABF8
:10DE50004FF0FF3061074FF0000102D40DE008F1F0
:10DE600001018846B9420FDA8045F8DB1AF808103C
:10DE70000029F4D108E008F1010188468142FADB6B
:10DE80001AF808100029F6D105985B46A0EB0807A0
:10DE900021463846179A00F09EFA284400EB080500
:10DEA00007E04DE02BE10DE01AF8010B5A461799F7
:10DEB0009047B8F10108F7D25B4621463846179AD9
:10DEC00014E142E00A220092C4F302524FF0000A29
:10DED000022A08D059F804CB032A4FEAEC710AD081
:10DEE0000DE029E02AE009F1070121F00702F2E83C
:10DEF00002C1914609E00FFA8CFC4FEAEC71042A4A
:10DF000003D14FFA8CFC4FEAEC71002907DA0A467C
:10DF10000021DCF1000C61EB02012D2202E0220560
:10DF200004D52B228DF80420012203E0E20701D062
:10DF30002022F7E7904653E00A2102E010220DE08C
:10DF400010214FF0000A00910BE010224FF0000A60
:10DF500044F004040827009203E008224FF0000A6E
:10DF60000092C4F30252022A05D059F804CB0021D2
:10DF7000032A08D009E009F1070121F00702F2E8BD
:10DF800002C1914605E01FFA8CFC042A01D10CF075
:10DF9000FF0C4FF00008220722D5702827D0009BE5
:10DFA00083F0100353EA0A0309D15CEA010206D0A8
:10DFB00030228DF804208DF8050002229046009B47
:10DFC00083F0080353EA0A030AD15CEA010201D193
:10DFD000620705D530228DF804204FF001087F1E1E
:10DFE000582809D037A003900EA8029013E04022D1
:10DFF0008DF804200122E1E737A0F4E7534660469C
:10E00000009AF6F7B9FC84460398825C0298A0F166
:10E010000100029002705CEA0100EFD1029806A9AB
:10E02000A1EB000000F1200A600702D524F480343F
:10E0300000E00127574502DDA7EB0A0000E00020C1
:10E0400000EB0A01009005984144A0EB0100059007
:10E05000E00306D45B462146179A059800F0BBF909
:10E060000544002706E001A85A46C05D179990476D
:10E070006D1C7F1C4745F6DBE0030CD55B46214653
:10E08000179A059800F0A7F9054404E030205A4695
:10E09000179990476D1C0099481E00900029F5DCE7
:10E0A00008E0029802995A460078491C0291179993
:10E0B00090476D1CBAF10001AAF1010AF1DC6BE195
:10E0C000092801003031323334353637383961624E
:10E0D0006364656600000000303132333435363712
:10E0E00038394142434445460000000000F060F9E1
:10E0F000054406F10106307800287FF4E9AD19B037
:10E100002846BDE8F08F620700D4062709F1070210
:10E1100022F0070CFCE80223E14603F000485FEA26
:10E12000080C02D00FF27C2C0DE05FEA045C02D5F3
:10E130000FF2742C07E05FEAC47C02D00FF26C2C63
:10E1400001E0AFF2700C4FF0FF3823F00043CDF840
:10E1500050C065280CD006DC452809D046281DD0C3
:10E1600047283ED13EE0662818D0672839D139E0EB
:10E170000021112F01DB112000E0781CCDE9000106
:10E1800006A90EA8FFF7CAFCDDE90F010E9A03915C
:10E190000021009207F1010A04914EE04FF0004087
:10E1A0000097CDE9011006A90EA8FFF7B7FCDDE93D
:10E1B0000F0203920E9B11990022DDF80CA0009330
:10E1C000049219B907F1010100EB010AB7EB0A004B
:10E1D00004D4C0F1FF3007F1010A0490AAEB070054
:10E1E000019046E0012F00DA01270021112F01DD07
:10E1F000112000E03846CDE9000106A90EA8FFF77E
:10E200008DFCDDE90F010E9A03910021049100922B
:10E21000BA4621070CD40399514500DA8A46BAF16F
:10E22000010F05DD009AAAF10101515C302908D0E7
:10E23000B84202DA10F1040F06DA0121CDE901102B
:10E2400017E0AAF10101E9E7002805DC049901447F
:10E250000491AAEB000102E0411C514500DD8A4611
:10E260000499A0EB010000F1010001904FF0004083
:10E270000290200704D40198504501DBCDF80480BA
:10E2800000208DF84F0002980DF14F07B0F1004FBC
:10E2900025D02B200E9002984FF0020800280CDAAF
:10E2A000404202902D200E9007E00A210298F6F7D6
:10E2B0004DFB3031029007F8011DB8F10001A8F1C3
:10E2C0000108F2DC02980028EFD1791E0E98087040
:10E2D000307800F0200040F0450007F8020D12A849
:10E2E000A0EB070000F107081498007800B10120A6
:10E2F00000EB0A01019801EBE07105984144A0EBA5
:10E300000100A0F101000590E00306D45B46214620
:10E31000179A059800F05FF805441498007820B12A
:10E320005A461799904705F10105E00323D55B464E
:10E330002146179A059800F04EF805441BE0049812
:10E34000002807DBDDE90301884203DD0098405C1B
:10E35000179901E0179930205A46904704986D1C90
:10E36000401C04900198401E019004D12E205A4672
:10E37000179990476D1CBAF10001AAF1010ADEDC81
:10E3800005E017F8010B5A46179990476D1CB8F134
:10E390000001A8F10108F4DC5B462146179A0598B4
:10E3A000A4E600002D0000002B000000200000006B
:10E3B0002DE9F041044600251E461746880405D481
:10E3C00006E039462020B04705F10105641EF8D566
:10E3D0002846BDE8F0812DE9F041044600251E469F
:10E3E0009046C80301D5302700E02027880405D5D2
:10E3F00006E041463846B04705F10105641EF8D5F0
:10E400002846BDE8F0814A68002A06D00A68531CF5
:10E410000B6010704868401E486070470A68531CC3
:10E420000B6010707047000008480068C0010BD5F1
:10E4300007480068C00707D00548803800680028F2
:10E4400002DA04490120087070470000FCED00E08A
:10E45000800E00E07C0100204FF06042D36F002B63
:10E46000FCD0436BD367D36F002BFCD0C07840EA5D
:10E470000120A2F87C0070474FF06041CA6F002A6B
:10E48000FCD081F87C0070472DE9F04780460D46AE
:10E49000680000F0F7F881464C46002715B90020C7
:10E4A000BDE8F08769004846F5F721FF00261CE02B
:10E4B00018F806007D2806D104F8010B012004F8A5
:10E4C000010BBF1C10E018F806007E2807D17D2044
:10E4D00004F8010B022004F8010BBF1C04E018F83B
:10E4E000060004F8010B7F1C761CAE42E0DB3A46C6
:10E4F00049464046F5F7E2FE484600F015F83D462D
:10E500002846CDE770B504460D46E1B20548FEF752
:10E5100010FD00BF40210348FEF73EFC0028F9D063
:10E52000204670BD0038014010B5002821D0114BA5
:10E53000001F0022196803E0814203D80A46496897
:10E540000029F9D152B11368841A9C4204D10068A1
:10E5500018441060104602E0506000E0186039B1C5
:10E5600002680B1A934203D10B681A44026049688F
:10E57000416010BD9401002010B5002100F008FE9C
:10E58000BDE8104000F0F4BD70B54FF4FA70F9F733
:10E59000F7F8FCF7CFFBFEF7D1FCFEF7A3FDFFF782
:10E5A00025F8F8F73BF8F9F7CBFAFDF70FFFFAF784
:10E5B000FDF9F6F74BFD4FF0FF3402E0F8F7CCFB26
:10E5C0000446002CFADBB4F5A57F07DA20A0FFF79C
:10E5D00059FA202023490860FDF76EFEF7F7F2FB99
:10E5E000F6F7FEFFFBF7ACFAF9F7DAFF1E48006812
:10E5F0006422B0FBF2F1B1F1807F00D31DE021F085
:10E600007F40401E4FF0E022506150170F2200283B
:10E6100007DA13071E0E154B00F00F052D1F5E5570
:10E6200003E013071D0E124B1D5400BF00204FF0D6
:10E63000E02290610720106100BFF5F789FD0D4AC7
:10E640000D490E48DFF838C000DF002070BD000023
:10E6500056425F4C6F772173687574646F776E0DE7
:10E660000A000000140C01405401002018ED00E0E5
:10E6700000E400E0B0190020010004004D8600080D
:10E68000D9F30008F0B50B30154D20F00701002438
:10E69000144A0FE003688B420BD38B4205D95E1AF4
:10E6A00043184768C3E9006700E04368136002C08D
:10E6B00004E0021D10680028ECD12046002802D199
:10E6C000286808B10020F0BD064A07481060074AD4
:10E6D000121A22F00702C0E9002401202860D7E7BF
:10E6E0009801002094010020043A0020003C002002
:10E6F00004460548036805480288214604A0FFF740
:10E70000C1F900BFFEE700004800002046000020DD
:10E710000D0A5B4F535F4572722025645D463D25AF
:10E72000642C4C3D2564000000BFFEE707480168EB
:10E730004FF0E0204161002181610721016104481F
:10E74000016841F07F41016040177047D0FA00082E
:10E7500020ED00E07047000010B50446012C0CD1FC
:10E7600000210648FDF79CFE0548007A28B90448B8
:10E77000407A10B901200349086010BD000800402C
:10E78000D8270020100C01400748007858B10748EE
:10E790000078401CC0B205490870032803DD002042
:10E7A00008700149087070474200002044000020B2
:10E7B0002DE9F34FA3B0814600201F9020902190B7
:10E7C00022901D901E9009900A900B900C900026AC
:10E7D000002400250690059000BF40210DA8F5F704
:10E7E00086FD0DA840F826906A210A20FDF70AF957
:10E7F00024E019F805002C281CD109A90598885592
:10E80000059818B900200DA941F8260000200590B0
:10E81000701CC6B209EB0500401C0DA941F826008A
:10E820000DA850F8260040782A2806D1012009A911
:10E83000885502E00598401C05906D1C249885427F
:10E84000D7D382210A20FDF7DDF8002424E00DA8AB
:10E8500050F82400FE49884206D30DA850F8241031
:10E86000FB48C830814216D30DA850F8240090B15F
:10E87000F8480078062805DCF6480078401CF54981
:10E88000087005E0F448807820F00100F2498870B3
:10E8900025B0BDE8F08F641C082CD8DB0D98E8B3D8
:10E8A0009DF824201FA80D99F5F74AFD1DAA062101
:10E8B0001FA800F0B3FF0D980088ADF87C00002081
:10E8C0008DF87E001FA8F5F775FE0830C0B20490E1
:10E8D0000A21049890FBF1F201FB1200C1B20791EA
:10E8E0006421049890FBF1F201FB12000A2190FBD5
:10E8F000F1F0C0B2089008980007000E0890089840
:10E9000000F0F0000890DDE907100843D249887252
:10E910009DF87500C8729DF8760000E000E008736D
:10E92000A4210A20FDF76EF80E9810B300201F9066
:10E930002090219022909DF825201FA80E99F5F790
:10E94000FFFC9DF87C0041280AD1C348807820F064
:10E950000100401CC04988700020BE4908700FE0CB
:10E96000BC480078062805DCBA480078401CB94944
:10E97000087005E0B848807820F00100B64988703A
:10E98000B2210A20FDF73EF8B348807810F0010F5D
:10E9900000D17DE70F98002854D0BC210A20FDF754
:10E9A00031F800201F902090219022901D901E9001
:10E9B0009DF826200DF17D000F99F5F7C1FC302060
:10E9C0008DF87C00C1210A20FDF71CF8052404E025
:10E9D0001FA9601C085C0855641C082CF8DB00208B
:10E9E0008DF884001DAA08211FA800F017FF002041
:10E9F0001F902090219022901098F8B19DF8272028
:10EA00001FA81099F5F79CFC9DF87C00532805D1B0
:10EA10009DF8740040F080008DF874009DF8770038
:10EA20009DF8761040EA01209DF8751040EA0140FB
:10EA30009DF8741040EA016087494861CF210A209F
:10EA4000FCF7E0FF1198E8B300201F902090219080
:10EA500022901D901E90D6210A20FCF7D3FF9DF82E
:10EA600028201FA81199F5F76BFC052404E01FA9C5
:10EA7000601C085C0855641C082CF8DB00208DF82D
:10EA800084001DAA08211FA800F0C8FEDC210A206E
:10EA9000FCF7B8FF1298A8B100201F902090219099
:10EAA00022909DF829201FA81299F5F749FC9DF89E
:10EAB0007C00572805D19DF8740040F080008DF847
:10EAC000740000E00FE09DF877009DF8761040EAB2
:10EAD00001209DF8751040EA01409DF8741040EA4D
:10EAE00001605D490861139800287DD0EA210A2061
:10EAF000FCF788FF00201F902090219022909DF825
:10EB00002A201FA81399F5F71BFC002505E01FA874
:10EB1000405D2E2800D104E06D1C9DF82A00A8421B
:10EB2000F5DC00BF9DF82A00401B401E0690F62130
:10EB30000A20FCF767FF032D14D19DF87C103039B3
:10EB4000642251439DF87D20303A02EB820201EBB2
:10EB500042029DF87E1030395018F5F7CDFE074679
:10EB6000884618E0022D0ED19DF87D1030399DF8B1
:10EB70007C20303A02EB820201EB4200F5F7BCFE4A
:10EB80000746884607E09DF87C10A1F13000F5F7B4
:10EB9000B3FE074688460698002814DD1FAA691CA4
:10EBA000515CA1F13000F5F7A7FE2C4A2C4BCDE9C2
:10EBB0000001F5F7C0FD3A464346CDE90201F5F7FD
:10EBC00013FD07468846274A274B38464146F5F746
:10EBD000B2FDCDE90201F5F7A0FE1FFA80FA64202C
:10EBE0009AFBF0F0000200E011E00A219AFBF1F13B
:10EBF0000A2291FBF2F302FB131140EA01101146C5
:10EC00009AFBF1F201FB12A10843134988614FF40A
:10EC100087710A20FCF7F6FE149838B300201F9085
:10EC20002090219022909DF82B201FA81499F5F791
:10EC300087FB9DF87C003038642148439DF87D10A7
:10EC4000303901EB810100EB41019DF87E000EE0BF
:10EC5000A80E002070000020B01D00209A999999FC
:10EC60009999B93F6F1283C0CAA1FD3F19E03038AE
:10EC700008441FFA80FB64209BFBF0F000020A218D
:10EC80009BFBF1F10A2291FBF2F302FB131140EA24
:10EC9000011011469BFBF1F201FB12B1084313492D
:10ECA000C8614FF48D710A20FCF7ACFE1598D8B1FD
:10ECB00000201F902090219022901D901E909DF882
:10ECC0002C201FA81599F5F73BFB1DAA06211FA8AC
:10ECD00000F0A4FD9DF87400044948729DF8750089
:10ECE00008729DF87600C87100BFD1E5B01D002004
:10ECF00070B50446207824280BD16078472808D1C5
:10ED0000E078522805D120794D2802D16079432836
:10ED100000D070BDE01DF5F71FFBC5B22946E01D10
:10ED2000FFF746FD0120034908700020487000BF2E
:10ED3000EFE70000B01D002030B502460C46134638
:10ED400000250CB9002030BD00211CE0505C7D285E
:10ED500008D1481C105C012804D17D2003F8010B68
:10ED6000491C0EE0505C7D2808D1481C105C02282C
:10ED700004D17E2003F8010B491C02E0505C03F82B
:10ED8000010B6D1C491C601E8842DFDC2846DAE757
:10ED900050E8001F31B10B6840E80032002AF7D17B
:10EDA00008467047BFF32F8FFAE7000070B50D4695
:10EDB000002812D04FF6FF71084C884204D2226816
:10EDC0000146104600F010FA20684570044800F033
:10EDD000C3F8BDE8704000F0EBBA70BD68010020D8
:10EDE000CC3900200F4810B50D4942680E480B6819
:10EDF0000068934204D00A60CB88421E1A448A807D
:10EE00008A8880B282420AD100200860054800F05A
:10EE1000A3F80146BDE81040024800F009BA10BD51
:10EE200088010020CC3900207001002070B51A4DF7
:10EE3000E86800282ED0A88A401EA882002623E079
:10EE4000A06838B161684160606810B1A1688160F4
:10EE50006660A66010482146183800F0E9F9A08ADB
:10EE6000A8826078042804D10C49E08A0988084403
:10EE7000A0820120607084F82500E068E860E06806
:10EE800008B10561E6602661A88A002802D1EC6815
:10EE9000002CD5D170BD0000E439002070010020A5
:10EEA00070B504000FD00D4DA17801262868827836
:10EEB00091420CD900F0D8F9286846702046BDE888
:10EEC000704000F075BA064800F046F8F7E7667043
:10EED0002146BDE87040024800F0AAB96801002050
:10EEE000CC3900200321FFF761BF000010B50446B4
:10EEF000008B084320836278618B062A16D0052A8E
:10EF000017D1084215D001EA0002628388432083AA
:10EF1000204600F0B3F901206070022084F825003B
:10EF20002146BDE81040034800F082B931EA0002F2
:10EF3000ECD010BDCC390020814202D342688A4215
:10EF400001D80120704750E8002F0A6040E8001205
:10EF5000002AF8D1002070470146406842684A60A4
:10EF60000B780022022B05D0012B03D0032B01D0FC
:10EF70004260704743680BB199604260826070479D
:10EF800070B5044600201546207001226270A17001
:10EF900084F824106060A060E06020612062A0829C
:10EFA000E0822083608384F8250084F82600208D89
:10EFB00018B90548FFF7ECFE206329462046BDE856
:10EFC000704000F00FB80000E81F00200348002147
:10EFD000016003490988C180704700008801002052
:10EFE000CCFA000810B5028D920803D10F4A12889E
:10EFF000C2F38D02036B03EB8202530700D5121F8D
:10F00000403A4FF08073C2E90E1300234FEA030425
:10F0100042F823405B1C0E2BFAD3C3691362C26211
:10F020004163006B0249016010BD0000C8FA00088E
:10F03000A52E5AE22DE9F0410F4604464168002012
:10F0400004F10C0621B1617802291AD0A189A9B373
:10F05000A189E289914246D2218904EB81010F61A5
:10F06000D6E85F1F491CC6E8521F002AF8D1218943
:10F07000491C89B22181E289914200D12081BDE8F9
:10F08000F081074660702046FFF766FF80F8257024
:10F090002189054604EB8101C0690861D6E85F0F4C
:10F0A000401CC6E8510F0029F8D12089401C80B2CD
:10F0B0002081E18988420BD1278109E0FFE72046C2
:10F0C000FFF74AFF0546C0690421076085F825104F
:10F0D00001206870284600F0D1F82946BDE8F041CB
:10F0E000034800F0A5B8BDE8F0410320FFF700BBDE
:10F0F000CC39002070B51B480121026851700068AE
:10F1000000F0B2F8184D6C7817E000BF05EBC401B1
:10F1100048680278E2B1012A1FD000F0E1F8E878EF
:10F12000641C844200D100240F48801CD0E84F1F8B
:10F13000491EC0E8421F002AF8D1A8780028E5D16E
:10F140006C700A48FFF708FFBDE8704000F030B966
:10F15000098989B2FFF7CAFEE1E78968FFF76AFF0C
:10F16000DDE700006801002000270020CC390020E6
:10F170000548017811B101214170704703494FF0F2
:10F1800080500860704700008001002004ED00E01E
:10F19000F0B4144A941CD5784FEA0206D4E84F3FE5
:10F1A000AB4202D1BFF32F8F0EE05B1CC4E8473F98
:10F1B000002FF3D1D6E84F3F5C1CAC4200D10024B5
:10F1C000C6E8474F002FF5D1D4789C4205D902EB11
:10F1D000C302C2E90101F0BC7047F0BC0220FFF796
:10F1E00087BA000000270020104A10B5D368ABB1E1
:10F1F00013469B8A03E08CB12246A48A2344D46838
:10F200008B42F8D3C460D0600261C46804B120614D
:10F21000591A8182908A401A908210BD0024C460DD
:10F22000D060C91A02619182848210BDE439002045
:10F2300030B502780023022A03D0012A01D0032A24
:10F2400000D101238C7800E01046426812B1957815
:10F25000A542F9D24A6041601BB102B19160886059
:10F2600030BD0020FBE7000003494A6842600022ED
:10F270008260486070470000CC39002010B50169F9
:10F2800000290ED0C268CA60C36800223BB18B8AD5
:10F29000848A23448B82C3681961C26000E08A8239
:10F2A000026110BD816839B142684A604168002935
:10F2B00001D0806888607047054906E04A6882424C
:10F2C00002D140684860704711460029F6D1704766
:10F2D000CC39002002220270002242604180704737
:10F2E00010B5416879B1FFF737FE0446FFF7C6FF56
:10F2F00001206070032084F825002146BDE81040FD
:10F300000348FFF795BF4188491C418010BD0000AC
:10F31000CC39002010B5416889B1FFF71DFE0446C5
:10F32000032084F825002046FFF7A8FF2046FFF7BA
:10F33000B7FD05490020096881F8250002E04188F1
:10F34000491C4180002010BD6801002010B50C460A
:10F35000418819B1491E4180002010BD34B10A4ACC
:10F360004368116823B1FFF763FF07E0012010BD78
:10F3700041601368002159601168886007212046A8
:10F38000FFF714FDF2E7000068010020064800685E
:10F39000D0E90B10814203D300680449884202D0AF
:10F3A0000120FFF7A5B9704768010020A52E5AE299
:10F3B0000749022248604270064A1278002A05D0A6
:10F3C00006C98A4202D0C078FFF756B870470000DD
:10F3D000680100207C0100202DE9F0471646884690
:10F3E0008146FFF721F8002004463E4A3E4902E0EC
:10F3F00042F82040401C0B889842F9D33B48382201
:10F4000001883B48FEF738FC3A48008880B240F05B
:10F410000042394801683948FEF72EFC3848082276
:10F42000018838480068FEF727FC374FFF25374A28
:10F43000FD703C8500213846FFF7A2FD34480421C9
:10F440000170446033480170C46004618482F86ACA
:10F450002030F4F777FE3048314907600220787099
:10F460002E48047044700978C170FFF7AFFD2D4835
:10F47000016841F47F0101600068290601EA00206B
:10F480002849C0431439B0FA80F00968C0F1080077
:10F49000C1F30221814200DB481C2249091F0B688D
:10F4A0006FF08072824063F317020A60FFF73EF943
:10F4B0001D49002808600CDB1C49455400F01F0260
:10F4C0000121914040114FF0E02202EB8000C0F892
:10F4D0000011324641464846BDE8F047002300F09F
:10F4E00095B8000084270020C4FA0008E0FA00085C
:10F4F000181E0020C8FA0008E4FA0008E81F0020DF
:10F50000EAFA0008A80000209439002029E7000842
:10F51000CC390020E43900206801002000270020B9
:10F52000E8FA000820ED00E08401002000E400E09B
:10F530000C4810B50268012151700068FFF794FE75
:10F54000FFF750FC08480168491C0160FFF76EFC9A
:10F5500000F03CF80548FFF7FFFCBDE81040FFF75E
:10F5600027BF00006801002070010020CC39002076
:10F5700001480068704700007001002070B50D461A
:10F5800004000AD00F48006838B1FFF701FC0028DA
:10F5900004D00D49C5808A8804E0002070BD19465A
:10F5A0009B881A44A24202D20B68002BF7D10B6849
:10F5B000121B0360828008608A888388D21A8A803E
:10F5C00070BD0000A80000207401002070B50D4C33
:10F5D0002068002815D0A0880B4E401EA0800AE0AD
:10F5E000E888FFF7B9F8A888A08028682060294635
:10F5F0003068FFF7A1FCA088002802D12568002D03
:10F60000EED170BD74010020A80000202DE9F0416A
:10F610001E46174680460C4611F0FF0F00D14C1CC9
:10F620001A48FFF7B5FB05002DD0C4F30F202F6358
:10F630002885E1B242462846EE61FFF7A1FC01248D
:10F640001348144906E000BF00EB840252F8042C72
:10F6500022B1641C0A889442F6D9002400EB84008D
:10F66000E6B240F8045C0C48EE70007818B1012155
:10F670002846FEF7F1FE2846FFF712FC074800680F
:10F6800080F825602046BDE8F0810000181E0020AB
:10F6900084270020C4FA00087C01002068010020B3
:10F6A0002DE9F05F544DDFF848B1DFF848A1296833
:10F6B0004FF000084FF00509012610B1CA788242C8
:10F6C0003FD1474681F80180F4F73FFD2968C862C1
:10F6D000FFF75CFE2868B046046A18E06068A8B1CD
:10F6E0002046FFF739FC064680F82590FFF7C6FD57
:10F6F00086F8018031464148FFF79AFDA4F8028060
:10F70000A660316AE1603462E46800E0E468002CDD
:10F71000E4D12868C2780AEB820141F8047C016BCD
:10F720003748FFF709FC286807639BF8001011B100
:10F730000021FEF791FE33482968FFF7FDFB2F609B
:10F7400051E03149098888420ED80AEB800757F802
:10F75000045C4DB12846FFF7A5FD2846FFF78EFD56
:10F76000CA46B1462C6A1BE0FF20BDE8F09F6068E6
:10F77000A8B12046FFF7F0FB064680F825A0FFF76A
:10F780007DFD86F8019031461C48FFF751FDA4F835
:10F790000290A660316AE1603462E46800E0E468E7
:10F7A000002CE4D147F8048C44461548296BFFF738
:10F7B000C3FB2C639BF8000018B100212846FEF71C
:10F7C0004BFE29460F48FFF7B7FB0C48406882788C
:10F7D000094801688B789A4208D981F8019001683C
:10F7E0000648FFF725FD0020FFF75AFB0020BCE785
:10F7F0007C0100208427002068010020CC390020F3
:10F80000E81F0020181E0020C4FA00080248006803
:10F81000002800D0C0787047680100202DE9FE4123
:10F8200004460B46002000900190029000271E46DF
:10F830000021002507E0605C00F00F0828466D1CE1
:10F840000DF80080491CB142F5DB0020E054002196
:10F8500010E01DF80100000701F1010C1DF80CC0BB
:10F860004CEA1060BC4607F1010808F0FF0702F8F7
:10F870000C00891CA942ECDB0020D054BDE8FE81BD
:10F88000B7830D0AB7830D067AE0F06A7AE0F06A72
:10F8900036FC000830FC000833FC000863FC00085C
:10F8A00047FC00085FFC00086FFC000867FC0008CC
:10F8B0006BFC00083AFC000839FC00083EFC00081C
:10F8C00043FC000855FC00085AFC00084BFC0008EB
:10F8D00050FC00082BFC000826FC000872FC000805
:10F8E000D5FB0008DEFB0008E7FB0008F0FB000882
:10F8F000F9FB000802FC00080BFC000814FC0008DF
:10F900001DFC0008C8FB000854010000580100005D
:10F91000610100006A010000720100007A0100002C
:10F92000820100008A0100009C0100000B0F0A0503
:10F93000021907051119010547542B524D503A5031
:10F94000534E3D256C753B4D4549443D25733B4326
:10F950004E554D3D303030303030303030303B550A
:10F96000494D49443D303030303030303030303B1C
:10F9700049503D25642E25642E25642E2564000003
:10F9800041542B535953434D443D2E2F7573722FC1
:10F9900062696E2F6D417373697374616E74203088
:10F9A00020302070686F6E652D636C69656E742001
:10F9B00025642025642E25642E25642E25640D0AD9
:10F9C0000000000068596364C8CCAAA7A2ABA56E6A
:10F9D0006A568A57F4BBFEFA26212D290D093E3AB4
:10F9E00037320A07F7F2FBF5FFF61C181314F1FD86
:10F9F000F90C9F089A97929B959F121B152C282310
:10FA0000F92A2722242E67252F98FC75F8F33C3815
:10FA100033340304050F06017A7772626B83848E98
:10FA2000C4CB8782353F364F3D399C989394424FE3
:10FA30004641818D4D49717D7996919D99C3C41D33
:10FA4000CECA7F767C7873747E7B751E1A171F165C
:10FA5000111D47195DC7C2CBC5CFD1DDD94C48C6F2
:10FA6000C1CD61C9D78CFD88A1ADA9B1BDB98B85C8
:10FA70008F4B4586DCD8D3D4DED2DBD5DFD64344EA
:10FA80004E4AE747ACA8A3A4AEBA0DB7B2AFA6E4FE
:10FA9000EEEAE7E2E1ED0FE966616D69BBB5BFB67D
:10FAA000ECE80BE3525C656F5853540C5E5B555F9A
:10FAB000312F9A0B0B5A2B9E0289593B0E516CEB3E
:10FAC000DAE631F608000000C80000010500010078
:10FAD0007FA90300000000001027000005000000BF
:10FAE000CC01000018070000100034000D0A0000CF
:10FAF0000000000000000000000000000000000006
:10FB000000000000000000000000000000000000F5
:10FB100000000000000000000000000000000000E5
:10FB200000000000000000000000000000000000D5
:10FB30000000000000000000000000004900040078
:10FB400000404040404040404040414141414140F0
:10FB500040404040404040404040404040404040A5
:10FB60004005020202020202020202020202020234
:10FB70000220202020202020202020020202020239
:10FB80000202909090909090101010101010101091
:10FB9000101010101010101010101010020202029D
:10FBA00002028888888888880808080808080808E1
:10FBB00008080808080808080808080802020202DD
:10FBC0004000000041FB000833313030333030302A
:10FBD0003330303000333130303330303000333276
:10FBE0003030333030300033333030333030300069
:10FBF0003334303033303030003335303033303020
:10FC0000300033363030333030300033373030333B
:10FC1000303030003338303033303030003339302A
:10FC200030333030300052414343005341434300AE
:10FC3000544700444D00544D005241504E0042453F
:10FC4000455000524750005347500052434950001E
:10FC50005343495000524D495000534D49500052B2
:10FC60004D5000534D5000564552004241540050F3
:10FC70005354000094FC000800000020A001000084
:10FC8000EC4F0008D0FC0008A0010020603E0000FE
:10FC90000CDB000802420302381E6BFFFF05012245
:10FCA00013A4270A142044C941032702010916F9A5
:10FCB000D91809224F2D0102030404100906070870
:10FCC00009020406087B366E376918013800000007
:04000005080041317D
:00000001FF
